:100000000C9450060C946D060C946D060C946D06C1
:100010000C946D060C946D060C946D060C946D0694
:100020000C946D060C946D060C946D060C946D0684
:100030000C946D060C946D060C946D060C946D0674
:100040000C946D060C946D060C946D060C946D0664
:100050000C946D060C946D060C946D060C942A138A
:100060000C946D060C946D060C946D060C946D0644
:100070000C946D060C946D060C946D060C946D0634
:100080000C946D060C946D060C946D060C940C1477
:100090000C946D060C946D060C946D060C946D0614
:1000A0000C946D060C946D060C946D06AEA83FD3AF
:1000B00000408D14C8DA1281FFD922DB002EA6A4DD
:1000C000AF2001A00000000001001000014010045A
:1000D00011441144AA55AA55EEBBEEBBFEBFEFFB7F
:1000E000FEFFEFFFFFFFFFFF805540332A24201C57
:1000F000191715131211100F0E0D0C0C0B0B0A0A09
:10010000090909080808080707070706060606067A
:100110000605050505050505050504040404040494
:100120000404040404040403030303030303030398
:100130000303030303030303030303030202020293
:10014000020202020202020202020202020202028F
:10015000020202020202020202020202020202027F
:100160000202020202020201A14EE42707E63FDC7E
:10017000E5B47E966CF5469B5A1053115B127213D0
:100180009A14D41520178018F519801B231DDE1E24
:100190000080D87F627F9D7E8A7D297C7D7A8478ED
:1001A0004176B573E270CA6D6D6ACF66F262D75E52
:1001B000825A5A5B5C5C5D5E5E5F60606162626336
:1001C000646465666667686869696A6B6B6C6C6DA8
:1001D0006D6E6F6F70707171727373747475757604
:1001E0007677787879797A7A7B7B7C7C7D7D7E7E68
:1001F0007F7F8080818182828383848485858686D7
:10020000878788888889898A8A8B8B8C8C8D8D8D4D
:100210008E8E8F8F909091919192929393949495CA
:1002200095959696979798989899999A9A9A9B9B4C
:100230009C9C9C9D9D9E9E9E9F9FA0A0A0A1A1A2D4
:10024000A2A2A3A3A4A4A4A5A5A6A6A6A7A7A8A85E
:10025000A8A9A9A9AAAAABABABACACACADADADAEED
:10026000AEAFAFAFB0B0B0B1B1B1B2B2B3B3B3B47F
:10027000B4B4A00318605F7DEA2B9364AA2E000338
:10028000C045D1011451C411600084102000836066
:100290002E3AE803B326B53A9C7CBD4ABF5EF062B5
:1002A000BB6EBD7E4001600144454A295111B02218
:1002B000AE378F3EBF2A2E2A3F3ABF469F42AE5AE4
:1002C0009F7CF147327A9F6C3F041F7DDF7D2E3A81
:1002D0009F226E3E9F2EAD5AF0433F7C7E785F7C1E
:1002E0009B6CF860B366E047980CF1030822210488
:1002F0000022E447E003F11386300A0004A404144A
:100300000670551F551E56BE745C55E2541FB41F2F
:100310000280398980290888227637882235384733
:1003200076788683051843885445132800000A0010
:1003300045C4C5C4254045242544E544C524E540BD
:1003400045C0452003C0374372355416300602C8F5
:1003500042528039342900000700350CE5ECE52CC9
:1003600003062515F505F524058024186545363561
:100370001235446301A08803020000000C00260A25
:10038000360A460A440B450AC40B451D5420B420C6
:1003900055006407A40702C047B87A85370004C82F
:1003A00078555676A76912967346016400001000CE
:1003B000B52C054C452CB501155F552094070477E5
:1003C0007497F504B5BC45BCB5B155B1A49705D635
:1003D0001480868848447457553333228997676F51
:1003E0006E9F73F498E3864551423037E6C340412F
:1003F00087D8A503A35C2B5B5D4100000800450581
:10040000C50BB504550C1606F60AA601660F02C008
:100410000A4657021300000008004505C50BB50445
:10042000550C1606F60AA601660F02C0A046570232
:1004300013000000D004BF04950486047D047204F8
:1004400061044404A5FF01B18001D5D001B1800150
:10045000D5D001C98001D58001C98001E1800100AA
:1004600000A5FF01B18001D5D001B18001D5D00137
:100470000000D5F001D5D001C9B0010000A5FF01F1
:10048000310149010000BD80025D016901E9A0015F
:10049000E9C0020000D9C002BDF002CDC002D9F00F
:1004A00002BD80024D025D01DDA001DDC001DDD095
:1004B00001DDE001DDF001DDF801DDFC020000BD41
:1004C0008001C9FF01310119010D01998F0100005F
:1004D000C9F002C9D002BDB001B19001A5800119D7
:1004E000010D010101000014050C050405EF0411C4
:1004F0001B09081C0A1D14120D0E13150A1D0F10DE
:100500001B141EFF020005060C0405FF070B16173F
:1005100018191AFF00010203040506020702080267
:1005200009020A020B04060C0D020E020F02100251
:1005300011001202130214001502FFEE07E207DA9F
:1005400007CE07C207B207A6074A073E07320716BB
:1005500007BA06AE06A20696068E068606720666DE
:10056000065A0646062E061606FE05E605CE05B612
:1005700005A20596057A057905FF0000001E14F412
:10058000055A1500087813FA0278140C052815FA94
:100590000878FF0000000000001E1500083CFF0066
:1005A00000000000001E13FD025A14060578150015
:1005B0000878FF0000000F0C0600160C0200100F58
:1005C00002001009025018000514FF0000000F0679
:1005D000060016060200100902001003025018005F
:1005E0000514FF0000000FF4060016F4020010F7D7
:1005F000020010F1025018000514FF0000000F095E
:10060000060016090200100C020010060250180025
:100610000514FF0000000F00060016000200100382
:10062000020010FD025018000514FF000000000039
:1006300000780EF400780E0C00780EFA00780E06A2
:100640000078FF0000000000001E0B01020004F60D
:100650000000030A0078FF0000000000001E8D0863
:1006600004B4FF0000000000001E0DF804B4FF00F9
:1006700000000000001E0B00020003F60000010A4B
:100680000078FF0000000CF40078FF0000008C0CE4
:100690000078FF0000000000001E15F6083CFF0077
:1006A00000000000001E150A083CFF0000000000CA
:1006B000001E1300021EFF000000000000780F0063
:1006C0000600160002001003020010FD02780F065B
:1006D00006001606020010090200100302780FFA45
:1006E000060016FA020010FD020010F702780F0350
:1006F00006001603020010060200100002780F0028
:100700000600160002001003020010FD0278180017
:100710000578FF0000000000002804F60014010A1C
:10072000003C03000028030A002804FE00A0FF008C
:1007300000000000001E0BF80278FF00000000001F
:10074000001E0B080278FF00000000000078110076
:100750000600170002001206020012FA02781106C3
:10076000060017060200120C02001200027811FAAD
:10077000060017FA02001200020012F402781109B2
:10078000060017090200120F02001203027811007E
:100790000600170002001206020012FA0278180082
:1007A0000578FF0000000000001E13F6021EFF0087
:1007B000000005F6003C060A006401000078FF0016
:1007C00000000000001E130A021EFF0000000000CF
:1007D000003C03F600A0FF00000000000078FF00CE
:1007E00000000000003C030A00A0FF000000000021
:1007F00000F0FF00000005004502550575012504C5
:10080000150702989AA9A99A214031000000A6A7CD
:10081000FFDDAA807F771582000000000000B00095
:1008200000B80600B83E0018BE0018B802188006CE
:1008300038000E30001CB00018A00618883E18388A
:10084000BE1CB8B01EB0861E803E0E00BE0000B0BA
:100850000600A01EB8BE1EB8BE1EB81E00B0060020
:10086000883E0038BE00B8B006B0861E883E1E38EE
:10087000BE18B8B006B0861E803E1E00BE1800B876
:100880000200800608000E38001CB80018B00618D8
:10089000803E1800BE1CB0B01EB8861EB83E0E3892
:1008A000BE0018B80218800618000E38000CB800F8
:1008B0001CA00618803E1800BC18B8B01EB8821ED6
:1008C000B8061E180E18181C0018B81E18B81E38C6
:1008D000B81EB81800B01E00803E0020BE00B8B0A0
:1008E00006B8861EB83E1E18BE1818B80618981E00
:1008F00038181E301818B01800A01E00883E0018C6
:10090000BE0018B80618801E18001E380018B8005F
:1009100000B80600983E0018BE0018B80610801EE9
:1009200000001E00001830000038000038000018D9
:10093000300018B80018B80638B80E30181EB01CB1
:100940001CA01E18801E18001E1800081C00001C89
:1009500000001C000008000000000000BE09BE09E5
:10096000AB09B509A409A4099D099D09485454502F
:100970003A2F2F535441524455494E4F2E43410074
:10098000284329205354455048414E4520484F4361
:100990004B454E48554C4C20323031390048494780
:1009A0004820200053434F52452000415544494FB1
:1009B000204F464600415544494F204F4E00535466
:1009C000415254005354415254494E4720424F4FD4
:1009D000544C4F414445522E2E2E00436C6173738C
:1009E000696300040015C545CCB5CF0560038025BB
:1009F00006233211030000080004B664BDA4BD053F
:100A00006045DC55DE54BD451E0180291304883441
:100A1000A643A557746431705600000B0304740498
:100A20007404740474346234623462346234DC34C6
:100A3000DC34DC34DC05AB05AB05AB05AB04E6040C
:100A4000E604E604E604790479047904795532452C
:100A5000244515452275DD75CF65C075CE760266D5
:100A60000336E5460336BE36BF26BF36BE55BD4506
:100A7000BF45A045BE0A889329624544793279670B
:100A800066A279682A291578462314401251302528
:100A90000002C8464672167612000002FA020808E2
:100AA0000805000000008B22EC25042E03184018D6
:100AB000FF0000000000000000042E03304030FF63
:100AC0000000000000000000042E03188018FF0042
:100AD00000000000000000042E03308030FF000002
:100AE000000000000000042E03182018FF00000082
:100AF0000000000000042E03302030FF0000000042
:100B0000000000000818040808080100000000DCCC
:100B10001F2C1F10FC030404040100000000DC1F54
:100B20002C1F007F0C0404048000000000151D35FC
:100B30001D20F607101010FF00000000000000004C
:100B4000015803202020030F3C050000002731013D
:100B5000F709202020031E78050100000000011B7A
:100B60000A202020061E2D0C030000000041E3098E
:100B7000080820030000000200000000047C0310AD
:100B80001010FF000000000000000004120C08100C
:100B900010FF0000000000000000047C0320101083
:100BA000FF000000000000000004120C101010FFF5
:100BB000000000000000000004AE03101010FF0051
:100BC0000000000000000004AE03202820FF000009
:100BD00000000000000004AE03304030FF000000C1
:100BE000000000000080120C101010FF0000000038
:100BF0000000000080120C201010FF000000000018
:100C000000000000120C101010FF00000000BD1DBD
:100C10000000000000005C0C450C1C0C05010000ED
:100C200000000000000000000000000000000000C4
:100C3000000000F406F6F008ECF406E20004D80424
:100C400002D80000D80202000000002004001808AA
:100C500000180C00101400001C0000240401000007
:100C60000F00000F00000F00000F00000F0C100518
:100C70001010FB1410F11808E71C04E21804E20736
:100C8000000540940C940405047404740C05C0021F
:100C900080AA0564120290AAAA0362340000000030
:100CA00011241FBECFEFDAE0DEBFCDBF11E0A0E020
:100CB000B1E0ECECFDE602C005900D92AE31B1075B
:100CC000D9F729E0AEE1B1E001C01D92A632B2072A
:100CD000E1F70E9430080C94E4360C940000FFFE0B
:100CE000FCF8F0E0C080000103070F1F3F7F209158
:100CF000170230911802422F430F203830F0403451
:100D00000CF00895342F222705C0403818F011F058
:100D100030E8321B31300CF408952F923F924F92FD
:100D20005F926F927F928F929F92AF92BF92B32EFB
:100D3000CF92DF92EF92FF920F931F93CF93DF93A7
:100D4000AFE2B2E0220F111C220F111C220F111C66
:100D5000A20FB11D112450911D02520F5090190283
:100D600080901A022EED3CE0790126EE3CE039013C
:100D700000911B0210911C02EFE1F2E020911E0293
:100D8000E20FF11DC08084EC90E0C80EDD24D91E76
:100D9000E6EEF0E0EB0DF11D6491772737E0332E9E
:100DA000272F26950203000C111C352D310D0AF456
:100DB0003327303414F00C942907232E1203000C2F
:100DC000111C382D310D12F40C94290711F40C94D8
:100DD000290730340CF030E42316DCF51124F70138
:100DE000022C0320E00DF11D9490F301032E03204B
:100DF000E00DF11DA4902694269426943695369500
:100E00003695ED01C20DD11DF6015370E50FF11DB0
:100E10004490231641F49A20492090940880092098
:100E20000428088216C03219142C192090940880C6
:100E30000920012809923A9519F049923A95E9F763
:100E4000AA2839F0142C1A20A09408800A2001281E
:100E500008821896760F5395BA9411F00C94D00628
:100E60001124DF91CF911F910F91FF90EF90DF90B0
:100E7000CF90BF90AF909F908F907F906F905F903A
:100E80004F903F902F9008953F924F92E4E03E2E76
:100E9000442411C03F924F923324442443940BC006
:100EA0003F924F92E4E03E2E4424439404C03F928C
:100EB0004F92332444242F920F931F93CF93DF93A9
:100EC000EB01DA01F9012224442829F0662777276B
:100ED0001127992704C0688179811A819B812D91FE
:100EE0003D914D915D91022F032B042B052BF1F1C8
:100EF0000081006061F0049F600D711D121D921D44
:100F00005003700D111D921D110C1108910D0181DE
:100F1000006061F0039F600D711D121D921D049F02
:100F2000700D111D921D5003100D911D0281006066
:100F300071F0029F600D711D121D921D039F700DB7
:100F4000111D921D049F100D911D5003900D0381E2
:100F5000006061F00203700D111D921D110C11084B
:100F6000910D0303100D911D0403900DE30DF21D6F
:100F70006993799319939993815009F0A5CF11241E
:100F8000DF91CF911F910F912F904F903F90089537
:100F900023B19CB18FB1392F3074922F9071932B64
:100FA00082958F70982B80912B018F5F8C3009F484
:100FB00080E020912A01821751F0E0912B01F0E0AE
:100FC000E25EFE4F2FE59227908380932B010895D8
:100FD00020912E0190912A0180912B01981741F0C8
:100FE000E0912A01F0E0E25EFE4F808180932E01C5
:100FF00080912A018F5F8C3009F480E080932A0170
:1010000090912E01822F8927982390932D0182237E
:1010100080932C01089587EE84B989EF85B980EC1F
:1010200087B918B880EF8AB990E29BB91DB890E4EF
:101030009EB910BA81BB8CE58CBD81E08DBD1EBC14
:101040001092720010927100EFE6F0E010821092A0
:101050006E001FBE1092D800108210928100089579
:101060000E940B0880EF0E94C6080E9457290E9428
:10107000C029FDCF0DB407FEFDCF8EBD08950DB480
:1010800007FEFDCF5C9808950DB407FEFDCF5C9A76
:101090000895AF92BF92DF92EF92FF920F931F934A
:1010A000CF93DF937C01EB010E9444082097A9F0C5
:1010B0008E01C131D10510F000E110E0C01BD10B51
:1010C0005701D02EF50181915F010E943A08DA9410
:1010D000D110F8CFE00EF11EE9CFDF91CF911F9133
:1010E0000F91FF90EF90DF90BF90AF900895CF9356
:1010F000C82F0E943F088C2FCF910C943A08CF93B1
:10110000DF93D82FC62F0E943F088D2F0E943A08E8
:101110008C2FDF91CF910C943A08AF92BF92DF925F
:10112000EF92FF920F931F93CF93DF937C01EB011C
:101130000E943F082097B9F08E01C131D10510F00F
:1011400000E110E0C01BD10BD02E5701F5018491B6
:101150000E943A08DA94C50101965C01D110F6CFDD
:10116000E00EF11EE7CFDF91CF911F910F91FF901D
:10117000EF90DF90BF90AF90089581E20E947708D2
:1011800080E00E9477088FE70C9477080F931F93F5
:10119000CF93C82F6AE070E080E090E00E940909D8
:1011A0005F9864E670E080E090E00E9409090E9488
:1011B00044085F9A6AE070E080E090E00E940909CC
:1011C00068E170E08CEA90E00E948D086C2F85ED5C
:1011D0000E947F080E94BD080E94440800E014E0BD
:1011E000C8010131110510F080E190E0081B190BD6
:1011F000C82F80E00E943A08C150D9F701151105A7
:1012000079F7CF911F910F91089560E074E00C94ED
:101210004908615071098109910948F020E23DE7D0
:101220003A950000E9F72A950000C9F7F2CF089532
:10123000CF93DF93EC019B01AC01BC0181E00E94E4
:101240004A07CE01DF91CF9108950F931F93FC01C0
:1012500080819181A281B381FB0100811181228172
:101260003381BC01CD01601B710B820B930B1F916D
:101270000F910895CF93DF9300D000D0CDB7DEB7A4
:101280009B01AC01BE016F5F7F4F81E00E944A0766
:1012900069817A818B819C810F900F900F900F90C4
:1012A000DF91CF910895AF92BF92CF92DF92EF92EC
:1012B000FF920F931F93CF93DF93CDB7DEB768975D
:1012C0000FB6F894DEBF0FBECDBFE42E2CE0829F98
:1012D000C00111249C0127563E4F6901590134E099
:1012E000A30EB11C8CE0689F8001112407561E4F8D
:1012F000B501C80104960E9425096D837E838F8302
:1013000098879CE0E99EA00111249A0127563E4F40
:101310007901B601C9010E94250969877A878B87FF
:101320009C87BE016B5F7F4FCE0109960E943A09F0
:1013300069837A838B839C83B501C70104960E94DD
:101340002509698B7A8B8B8B9C8BB601C8010E9417
:1013500025096D8B7E8B8F8B988FBE016F5E7F4FC3
:10136000CE0145960E943A096D877E878F87988BBC
:10137000BE016F5F7F4FCE010D960E9425096896D2
:101380000FB6F894DEBF0FBECDBFDF91CF911F9196
:101390000F91FF90EF90DF90CF90BF90AF900895A6
:1013A00061E0680F42E0480F90911102691708F060
:1013B000691B491708F0491B0C945309EF92FF92DF
:1013C0001F93CF93DF937C0110911102C9E9D1E003
:1013D000112341F0AE01BE01C7010E945C182C969A
:1013E0001150F6CFDF91CF911F91FF90EF900895AC
:1013F00010921302109215021092140208950E9486
:10140000DC1188E080931E028FE291E00E94A41715
:101410000C94F809CF93909111029A3070F5492FEE
:101420005CE0841710F5242F30E0B9016150710998
:10143000529FD001539FB00D1124A756BE4F569F07
:10144000F001579FF00D1124E756FE4FC52F019074
:101450000D92CA95E1F7FB01E157FE4F6081F9015A
:10146000E157FE4F60834150DCCFE82FF0E0E157B9
:10147000FE4F10829F5F90931102CF9108952F929B
:101480003F924F925F926F927F928F929F92AF9214
:10149000BF92CF92DF92EF92FF920F931F93CF9361
:1014A000DF93CDB7DEB766970FB6F894DEBF0FBEF9
:1014B000CDBF882E962E682E712C6CE0669DC001E3
:1014C000679D900D11248C0107561E4F1E8B0D8BAE
:1014D000042E000C550B9A01220F331F220F331FCD
:1014E00083E0440F551F8A95E1F7CA0180509F4F52
:1014F0009E878D87F801E20FF31F208031804280A4
:101500005380892D90E0699D200D311D1124F90132
:10151000E756FE4FE080F18002811381E98AFA8A62
:101520000B8B1C8BE218F30804091509ED82FE826F
:101530000F831887ED85FE8540815181628173811B
:10154000EF28E02AE12AA9F4E988FA880B891C89A6
:10155000E416F506060717070CF4C8C14481558147
:1015600066817781E416F506060717070CF0BEC101
:10157000C4C109891A892B893C89041715072607D4
:1015800037070CF068C0FC01E157FE4F80818111E4
:1015900062C091E0908390931202241635064606AD
:1015A00057060CF4AAC1892D0E940A0A981408F45F
:1015B00083949394ED85FE8580819181A281B3818E
:1015C00082199309A409B5096C017D01FF0CCC08AF
:1015D000DC2C76019C01AD016C2D7C2D8C2D9C2D7D
:1015E00000E10E94B736AD80BE80CF80D884ED8008
:1015F000FE800F811885110FEE08FE2C8701E98609
:10160000FA860B871C87E984FE2C0E2D1E2D0E9466
:10161000E23529833A834B835C83892D90E0ECE0AB
:10162000E89F9001E99F300D112427563E4FE89D19
:10163000A001112447565E4F0197E89FB001E99F32
:10164000700D112467567E4F8E010F5F1F4F83E090
:101650000E94561567C024163506460657060CF03C
:1016600061C081E080931202891420F4F301E157F4
:10167000FE4F808381E0880D0E940A0A891408F4D5
:101680009394ED85FE8580819181A281B381821939
:101690009309A409B5096C017D01FF0CCC08DC2C71
:1016A00076019C01AD016C2D7C2D8C2D9C2D00E1D3
:1016B0000E94B736AD80BE80CF80D884ED80FE809A
:1016C0000F811885110FEE08FE2C8701E986FA8636
:1016D0000B871C87E984FE2C0E2D1E2D0E94E235FF
:1016E00029833A834B835C8373010FEFE01AF00A7E
:1016F0008CE0899D9001112427563E4F8E9DB001AC
:101700008F9D700D112467567E4F8E010F5F1F4F06
:101710004D895E8983E00E945615F701E157FE4F1F
:1017200082E08083ED85FE8584819581A681B781E5
:10173000E988FA880B891C89E816F9060A071B074D
:101740000CF465C0E92DF0E0E157FE4F2081211136
:101750005EC021E0208320931202281639064A0633
:101760005B060CF0CAC0892D0E940A0A981408F47E
:1017700083949394ED85FE8584819581A681B781BC
:1017800082199309A409B5096C017D01FF0CCC08ED
:10179000DC2C76019C01AD016C2D7C2D8C2D9C2DBB
:1017A00000E10E94B7364D805E806F807884770CB0
:1017B0004408542C3201AD80BE80CF80D884E42C04
:1017C000F42C042D142D0E94E23529833A834B8397
:1017D0005C83892D90E0ECE0E89F9001E99F300D5B
:1017E000112427563E4FE89DA001112447565E4F15
:1017F0000197E89FB001E99F700D112467567E4F55
:101800008E010F5F1F4F83E00E94561576C0281689
:1018100039064A065B060CF470C081E08093120220
:10182000682C712C891420F4F301E157FE4F80835A
:1018300081E0880D0E940A0A891408F49394ED85CA
:10184000FE8584819581A681B78182199309A409B7
:10185000B5096C017D01FF0CCC08DC2C76019C01E4
:10186000AD016C2D7C2D8C2D9C2D00E10E94B73696
:10187000ED80FE800F811885110FEE08FE2C870188
:10188000ED86FE860F87188BAD80BE80CF80D88412
:10189000ED84FE2C0E2D1E2D0E94E23529833A8305
:1018A0004B835C8323010FEF401A500A8CE0899D23
:1018B0009001112427563E4F869DA001879D500D13
:1018C000112447565E4F849DB001859D700D1124F3
:1018D00067567E4F8E010F5F1F4F83E00E945615A3
:1018E000F201E157FE4F82E0808307C0FC01E1571F
:1018F000FE4F21E0208320931202892D66960FB6B9
:10190000F894DEBF0FBECDBFDF91CF911F910F9135
:10191000FF90EF90DF90CF90BF90AF909F908F900F
:101920007F906F905F904F903F902F900895CF934E
:10193000DF9350911102CFE8D1E029E931E090E046
:1019400080E04CE09517B1F06881613071F0891743
:1019500059F0489FD0011124A756BE4FF901642FBA
:1019600001900D926A95E1F78F5F19929F5F245F56
:101970003F4FE8CF80931102DF91CF9108952F92CE
:101980003F924F925F926F927F928F929F92AF920F
:10199000BF92CF92DF92EF92FF920F931F93CF935C
:1019A000DF9300D000D0CDB7DEB783E022242A94A5
:1019B000280E882309F46EC0109212028091110241
:1019C000815060E090911102691730F4422D0E941D
:1019D0003F0A61E0680FF6CF80911202882381F000
:1019E0000E94970C211002C0822DE0CF909111022D
:1019F000EFE8F1E080E0891719F011928F5FFBCFDB
:101A000082E02812F1CF312C80911102381660F754
:101A1000832C912C9CE0989D3001999D700C112491
:101A2000F301E756FE4F2F0180859185A285B3858E
:101A30000097A105B10561F1AC01BD01770F440B21
:101A4000542FBA015C016D01E42EF42E042F142FE3
:101A500020E030E040E050E061E070E080E090E0C5
:101A60000E94E23529833A834B835C83BE016F5F1A
:101A70007F4FC2010E941809BE016F5F7F4FC301F3
:101A800083569E4F0E941809F401E157FE4F1082C1
:101A90003394BACF0F900F900F900F90DF91CF91AA
:101AA0001F910F91FF90EF90DF90CF90BF90AF907C
:101AB0009F908F907F906F905F904F903F902F906E
:101AC00008950F931F93262F30E044E0649F800D0C
:101AD000911D1124FC014081518162817381C901F2
:101AE000880F991FF3E0220F331FFA95E1F7F901F0
:101AF000E050FF4F0081118122813381401751074F
:101B0000620773079CF0FC01EE0FFF1FEE0FFF1F33
:101B1000EC5FFE4F81E00081118122813381041747
:101B20001507260737071CF080E001C081E01F91F0
:101B30000F9108955F926F927F928F929F92AF92D2
:101B4000BF92CF92DF92EF92FF920F931F93CF93AA
:101B5000DF9320919F013091A00180911102E9E96A
:101B6000F1E0590191E0612C712C981778F44289C9
:101B700053894217530714F4792E9A01A416B50617
:101B800014F4692E5A019F5F3C96EFCF2A153B054E
:101B900009F452C11FEF170D91E0970D092F17FDA2
:101BA000180F682F70E0492F092E000C550B4617AF
:101BB000570714F0092F081B572C4CE01403F001B1
:101BC0001124E356FE4F0280F381E02D2E173F07CC
:101BD00011F05CE014C09FEF910F97FD03C0512EF0
:101BE000192FECCF980FFBCF91E0900FE92F092E22
:101BF000000CFF0BE617F7077CF4702E092F4CE062
:101C00000503F0011124E356FE4F0280F381E02D1D
:101C10002E173F0749F302C0981BEFCF552D5403F1
:101C2000F0011124E756FE4FE281672D6403D001D5
:101C30001124A756BE4F12964C914E170CF058C067
:101C40008E2FE42F482F54C0672D6503C001112447
:101C5000DC01A756BE4F1296FC91DC01A356BE4F85
:101C600012968D919C911397B701681B790BC1F067
:101C7000D601A81BB90B9A2F80E00E947135DB01B9
:101C80008D2FDD0F990B8F1B9109F7FD9395A89F61
:101C9000B001A99F700DB89F700D1124DF2FD70FD1
:101CA00046012815390509F079C0A814B90409F4CA
:101CB000C3C0101709F4C0C0B0E88B1691040CF033
:101CC000BBC08C149D0409F09CC0611609F49CC033
:101CD0008FEF810F87FF03C090911102890F8E143F
:101CE0009F0419F4601296C0762C512E182F94017F
:101CF0005CE01503B0011124DB01A356BE4F129620
:101D0000CD90DC9013970503C0011124DC01A3568C
:101D1000BE4F1296ED90FC901397DB01A756BE4F75
:101D20001296CC91DC01A756BE4F1296DC91CE14D0
:101D3000DF040CF489CFCE14DF0409F4B1CF5CE0EA
:101D4000652D6503C0011124DC01A756BE4F129614
:101D5000FC91DC01A356BE4F12968D919C91139776
:101D6000B601681B790BC1F0D701A81BB90B9A2FDC
:101D700080E00E947135DB018C2FCC0F990B8F1BFB
:101D80009109F7FD9395A89FB001A99F700DB89F89
:101D9000700D1124CF2FC70F470183CF18141904DA
:101DA0000CF083CFDC171CF48C2FCD2FD82F6C2F89
:101DB0006E1B5D2F541B842F8E27082E000C990B51
:101DC000762F752B872B892BC9F08D2F842387FDC8
:101DD00015C0E03414F0C0348CF420931702882D21
:101DE000821B80931802E09319024F5F40931A02FE
:101DF00060931B0250931C020E9477064D2FEC2F1C
:101E000054CF812F152D6BCF862D162D8E149F0448
:101E100009F06BCF91E0900F20911102A92F092EAC
:101E2000000CBB0B622F70E0702E092FA617B707AE
:101E30000CF45BCF021B59CFDF91CF911F910F9113
:101E4000FF90EF90DF90CF90BF90AF909F908F90DA
:101E50007F906F905F900895CF92DF92EF92FF9204
:101E6000CF93C09111028FEF8C0F843008F07CC0AB
:101E7000C13061F560E089E991E00E94610D811156
:101E800073C061E089E991E00E94610D81116CC02D
:101E900062E089E991E00E94610D811165C0809145
:101EA0009F01805C80931702C093180280919B0170
:101EB00090E2980F909319028F5D80931A02CF9150
:101EC000FF90EF90DF90CF900C9477060E94BF0CAC
:101ED00080911102833030F430911102E9E9F1E090
:101EE00020E031C080E00E94D0096B017C01C1E09C
:101EF00080911102C81748F48C2F0E94D009C60E99
:101F0000D71EE81EF91ECF5FF3CFC094D094E094A3
:101F1000F094CC24F7FCC394DD24EE24FF248091BC
:101F200016028C1121C0D8CF828193818096938331
:101F3000828386819781805C9F4F97FD07C097833E
:101F400086832F5F3C963213EFCF05C01482158233
:101F500016821782F6CF333038F0CF91FF90EF9092
:101F6000DF90CF900C949A0DCF91FF90EF90DF907F
:101F7000CF9008952F923F924F925F926F927F92EF
:101F80008F929F92AF92BF92CF92DF92EF92FF9289
:101F90000F931F93CF93DF93CDB7DEB7C554D1090D
:101FA0000FB6F894DEBF0FBECDBF7C0180E3EFE239
:101FB000F1E0DE01119601900D928A95E1F7AE01F4
:101FC0004F5F5F4F6FE571E08FE291E00E94AF17C6
:101FD0000FE211E061E676E0C8010E94180961E6AF
:101FE00076E0C80104960E941809F8018081918169
:101FF000A281B38144815581668177814083518379
:102000006283738384839583A683B783045F1F4FA2
:10201000F1E00F351F07F1F68E010C5C1F4F40E019
:10202000B701C8010E941B12C8010E9466122CA9A8
:102030003DA93AAF29AF292F2F7099249394920E7E
:10204000492D50E05CAF4BAF9927880F991F849FB3
:102050009001859F300D949F300D112489AD9AAD6C
:10206000820F931F9DAB8CAB25960FAF25972696BD
:102070001FAF269725968FAD259726969FAD26975D
:102080000E946612009709F466C1582F5F7358AF1B
:10209000292F269526952695E22FE7702E2E6C0186
:1020A00044E0D49EC12CDD241124C39456E09695BF
:1020B00087955A95E1F78F7199274BAD5CAD849F59
:1020C0005001859FB00C949FB00C1124AA0CBB1C2E
:1020D00089AD9AADA80EB91E8CA99DA9AEA989ABF0
:1020E0009AABABAB98ADE92EF12C20FF02C0EE0C01
:1020F000FF1C21FF02C0EE0CFF1C22FF02C0EE0CF1
:10210000FF1CB701CE01C1960E948B12C701E8AD3A
:10211000EC9D800D911D112403967C01F694E794AB
:10212000F694E794EE0CFF1C8CA99DA99C012E0D42
:102130003F1D21963FAF2EAF219731E0309316021D
:10214000D12C49A85AA88BA848AD4FAB5D2D517032
:1021500022965FAF22978D2D827023968FAF2397A3
:102160009D2D947024969FAF2497EFA9E150EFAB7B
:10217000EF3F09F4C0C0C0921102ECA9FDA98491FF
:102180002EA990E0022E02C0959587950A94E2F759
:102190008F7094E092279EAB911103C03196FDABF6
:1021A000ECAB80931E022FE831E03EAF2DAFB9E9D2
:1021B000EB2EB1E0FB2E312CF201649170E0082C83
:1021C00002C0759567950A94E2F76F70F4E08F2668
:1021D00019F42FEF421A520A90911302969E300181
:1021E000112480911502B301680F711D660F771FCE
:1021F0006A0D7B1D992351F1C7010E94D016809171
:102200001402B301680F711D660F771F6A0D7B1DE5
:1022100037013CE0630E711CC3010E94D01680910F
:10222000130290E0A0E0B0E0BA2FA92F982F8827E2
:1022300089839A83AB83BC838E010F5F1F4F930109
:10224000A701B70183E00E94561503C0C7010E9491
:10225000D01622964FAD2297442381F0F70180815A
:102260009181A281B381B095A095909581959F4F62
:10227000AF4FBF4F80839183A283B3832396FFAD7B
:102280002397FF2381F0F70184819581A681B7818F
:10229000B095A095909581959F4FAF4FBF4F848388
:1022A0009583A683B7832496FFAD2497FF2381F0FF
:1022B000F70180859185A285B385B095A09590950D
:1022C00081959F4FAF4FBF4F80879187A287B3877C
:1022D000EDADFEAD1192FEAFEDAF3394FCE0EF0E2D
:1022E000F11C3C1408F468CF8FE291E00E94DE09F3
:1022F0000E942C0F3ACFD21431F1822D91E0882325
:1023000061F080FD03C0990F8695FBCFD926292F58
:102310002D2119F4990F8695F2CF8D2D90E0AC0107
:10232000559547959C0135952795359527952427F3
:102330003527822793278170992721E08227817092
:1023400080931602FECE21964EAD5FAD21975DAB18
:102350004CAB1EAA8FCECB5BDF4F0FB6F894DEBF1F
:102360000FBECDBFDF91CF911F910F91FF90EF90E6
:10237000DF90CF90BF90AF909F908F907F906F90A5
:102380005F904F903F902F90089590E1893020F01A
:10239000292F281B822FFACF880F880F460F64172A
:1023A00039F0E62FF0E0E15EFD4F80836F5FF7CFFD
:1023B000089541E00C94C511EFE1F2E080E094E073
:1023C000899F900111242193883009F481E08F5F67
:1023D00092E0EF32F90799F780915D0690915E06E1
:1023E00069E08F700E94D91180915D0690915E0620
:1023F00080FD02C086E001C083E06AE00C94D91140
:102400000C94DC1180911D028F5F837080931D02FC
:102410000E94BD088FE292E00C940509FC019281B4
:1024200084E089278283811105C080819181019692
:10243000918380830895FC0171836083842F880FCA
:10244000880F828343FF04C06F5F7F4F7183608377
:102450000895FF920F931F93CF93DF93DC011296A1
:10246000FC901297ED91FC911197FF2021F18C01C6
:10247000C4910E940E12D801ED91FC911197E49144
:10248000F0E012960C9002C0F595E7950A94E2F7F9
:10249000DE2FDF70C8010E940E12EC2FF0E002C0A8
:1024A000F595E795FA94E2F7EF708E2FB0E1DB9F98
:1024B000800D112405C0CF0101968D939C938491CA
:1024C000DF91CF911F910F91FF9008951F93CF93AC
:1024D000DF93DC0112968C911297882371F0ED0145
:1024E000CD010E942912182FCE010E94291290E0DE
:1024F000982F8827810F911D0AC08D919C9111976B
:10250000FC012591349102968D939C93C901DF9132
:10251000CF911F9108959B0136952795FC0140812D
:102520005181240F351F3183208360FD0C940E12DE
:102530000895DC0112961C92129713961C92139721
:10254000E62FF0E0EE0FFF1FEC5CFB4F85919491BE
:1025500011969C938E9381E012968C9308958091AE
:1025600060068823E1F3109260060895E82FEF706B
:10257000EC3008F0E0E0F0E0EE0FFF1FE05DF94F17
:102580009FE8981B92959F7020813181A90102C01C
:10259000559547959A95E2F7CA010895282F6CE062
:1025A0000E94653594E0899F200D1124822F80526E
:1025B0000895BF92CF92DF92EF92FF920F931F93F5
:1025C000CF93DF93C8E4D6E080E5E82E86E0F82ECE
:1025D0008A818823B9F081508A83811113C0C88011
:1025E000D98086010F5F1F4FF601B490B1101CC057
:1025F000F70111821082F80184918A830F5F1F4FC7
:10260000198308832496F5E0EF0EF11C86E0C035AF
:10261000D807F1F6DF91CF911F910F91FF90EF90C6
:10262000DF90CF90BF9008958B8181508B0D8F7775
:102630000E94CE120E94B612F70191838083B7FEEA
:10264000DACFF2E0CF0ED11CF8010491F701048338
:102650008601D1CF1F920F920FB60F9211242F93A4
:102660003F934F935F936F937F938F939F93AF931A
:10267000BF93EF93FF930E94C80780912F068111AB
:1026800010C091E090932F06789480915F068F5F41
:1026900080935F06909360060E94D912F89410927E
:1026A0002F06FF91EF91BF91AF919F918F917F91F5
:1026B0006F915F914F913F912F910F900FBE0F90AF
:1026C0001F9018958F929F92AF92BF92EF92FF92B8
:1026D0000F931F93CF93DF9390935C0680935B06D9
:1026E0009C01990F440B550B60E072E18AE790E082
:1026F0000E9485351092710010926E0021153105EF
:1027000081E04807510518F1E3E056954795379564
:102710002795EA95D1F72115310581E04807510544
:10272000C0F073E056954795379527957A95D1F780
:102730002115310581E04807510568F062E05695A2
:102740004795379527956A95D1F784E005C081E0D4
:1027500003C082E001C083E010929000806180930A
:10276000910010929200309397002093960016BC2F
:1027700083E084BD85E085BD80905B0690905C061B
:102780008114910419F108E711E0C0E3D6E038E4C0
:10279000E32E36E0F32E092C000CAA08BB08F80142
:1027A00065917491CB01770FAA0BBB0B7727662736
:1027B000A50194010E948535299339930E5F1F4F1F
:1027C000EC16FD0661F781E08093710081E0809353
:1027D0006E007894DF91CF911F910F91FF90EF9051
:1027E000BF90AF909F908F90089580EC80935A0691
:1027F000E0E5F6E01182108216821582F89488E0F6
:10280000E8E4F6E0DF011D928A95E9F778940895EF
:102810000E9462130C94F5133F933FB73F934F937D
:102820005F936F93AF93BF93EF93FF93A0E5B6E0F1
:1028300042E050E860E0ED91FD913E2F3F2B11F416
:1028400013961CC03C913E0F3D933C913F1F3D931E
:10285000EC91E170ED9179F0E3233E2F3F703695D6
:10286000E295EF70F0E0E859FE4FE491EE0F3A95F3
:10287000EAF720F402C0E31B0AF4652750954150A3
:10288000D1F630915A06632368B9FF91EF91BF9159
:10289000AF916F915F914F913F913FBF3F911895DD
:1028A000FC0180819181A281B381181619061A0654
:1028B0001B060CF053C080389105A105B10544F109
:1028C00025E08115F2E09F07A105B1054CF062E01B
:1028D000B595A795979587956A95D1F72F5FF1CF15
:1028E000B595A79597958795E0ECE80FF0E0EE5445
:1028F000FE4FE4918E2F90E0A0E0B0E0BC01CD014E
:1029000004C0660F771F881F991F2A95D2F7089574
:102910002BEF42E0880F991FAA1FBB1F4A95D1F7E2
:102920002F5F80389105A105B1059CF3B595A7955A
:1029300097958795E0ECE80FF0E0EE54FE4FE491B8
:102940008E2F90E0A0E0B0E0BC01CD0104C09595D1
:102950008795779567952A95D2F7089560E070E09E
:10296000CB010895FC01462F50E060E070E0BA0111
:102970005527442780819181A281B3814817590747
:102980006A077B0764F070956095509541955F4F9D
:102990006F4F7F4F84179507A607B70724F440832E
:1029A0005183628373830895FC0140815181628168
:1029B000738177FF0BC070956095509541955F4F7F
:1029C0006F4F7F4F408351836283738308958F924B
:1029D0009F92AF92BF92CF92DF92EF92FF92FB0154
:1029E000CC24DD247601C21AD30AE40AF50A815008
:1029F000B8F080809180A280B380B7FE06C0C81472
:102A0000D904EA04FB0454F405C082169306A40614
:102A1000B50624F410821182128213823496E7CF15
:102A2000FF90EF90DF90CF90BF90AF909F908F90EE
:102A30000895CF92DF92FF920F931F93CF93DF936E
:102A400000D000D0CDB7DEB76A018B01F82EFF2091
:102A500001F1F60181919191A191B1916F01898369
:102A60009A83AB83BC83CE0101960E94D414F801F3
:102A700081919191A191B1918F01FA9449815A81EB
:102A80006B817C8184179507A607B70704F780E060
:102A900001C081E00F900F900F900F90DF91CF91C8
:102AA0001F910F91FF90DF90CF9008954F925F920A
:102AB0006F927F928F929F92AF92BF92CF92DF924E
:102AC000EF92FF920F931F93CF93DF9300D000D02C
:102AD000CDB7DEB75B0169014801843009F483E0BA
:102AE0007A01182F112321F1B701C6010E9425098F
:102AF00069837A838B839C83B401CE0101960E9403
:102B00003A09F70141905190619071907F01DC0189
:102B1000CB01840D951DA61DB71DF50181939193E1
:102B2000A193B1935F01F4E0CF0ED11C1150DACF25
:102B30000F900F900F900F90DF91CF911F910F91F9
:102B4000FF90EF90DF90CF90BF90AF909F908F90CD
:102B50007F906F905F904F9008950F931F93CF9346
:102B6000DF9300D000D0CDB7DEB7F901012E000C05
:102B7000220B330B322F212F102F002709831A83AA
:102B80002B833C838E010F5F1F4F9F010E945615C0
:102B90000F900F900F900F90DF91CF911F910F9199
:102BA0000895BF92CF92DF92EF92FF920F931F93FF
:102BB000CF93DF93B82EEB018A01BA01CE010E94B8
:102BC0003A096B017C01BA94BB2061F024960C5F3A
:102BD0001F4FB801CE010E943A09C60ED71EE81E4B
:102BE000F91EF1CFC701B601DF91CF911F910F916F
:102BF000FF90EF90DF90CF90BF900895CF92DF923B
:102C0000EF92FF920F931F93FB01815098F0DA012E
:102C10000D911D912D913D91AD01C080D180E2803B
:102C2000F3800C0D1D1D2E1D3F1D0193119321934B
:102C30003193EBCF1F910F91FF90EF90DF90CF90EA
:102C40000895CF92DF92EF92FF920F931F93FB01B3
:102C5000815098F0DA01CD90DD90ED90FD90AD01BE
:102C600000811181228133810C191D092E093F0930
:102C70000193119321933193EBCF1F910F91FF900B
:102C8000EF90DF90CF9008952F923F924F925F92F6
:102C90007F928F929F92AF92BF92CF92DF92EF92EC
:102CA000FF920F931F93CF93DF93782E4A01EB018E
:102CB0007A948FEF781669F188819981AA81BB8116
:102CC0006C017D01FF0CCC08DC2C76019C01AD0170
:102CD0006C2D7C2D8C2D9C2D00E10E94B736F401CB
:102CE000E080F1800281138117012801550C220830
:102CF000322C210157016801E22CF22C022D122DF9
:102D00000E94E235C901DA0189939993A993B99395
:102D1000CFCFDF91CF911F910F91FF90EF90DF9078
:102D2000CF90BF90AF909F908F907F905F904F908B
:102D30003F902F900895FF920F931F93CF93DF93AF
:102D4000CDB7DEB728970FB6F894DEBF0FBECDBF64
:102D5000F82E8B01AB010E94D1156D837E838F838A
:102D60009887CE0105960E94501469837A838B83DD
:102D70009C83672B682B692B39F0AE014F5F5F4F47
:102D8000B8018F2D0E94441628960FB6F894DEBF26
:102D90000FBECDBFDF91CF911F910F91FF9008958E
:102DA000FB0125913491422F4F70485FFC0154E0A4
:102DB000515001F1822F807F082E000C990B64E0A6
:102DC000959587956A95E1F7092E000CAA0BBB0B28
:102DD000042E04C0880F991FAA1FBB1F0A94D2F7A4
:102DE00081939193A193B19374E0369527957A9549
:102DF000E1F7DECF08959B01AC01BC018CE00C949F
:102E00004A070F931F93CF93DF93FC01DB018A01E5
:102E100080E3EF0119928A95E9F721112FC040E074
:102E200050E061E070E04083518362837383E80186
:102E3000488159816A817B81408B518B628B738B76
:102E400040A351A362A373A34D915D916D917C91B9
:102E50001397448B558B668B778B8D919D910D903D
:102E6000BC91A02DB095A095909581959F4FAF4FA7
:102E7000BF4F848F958FA68FB78F61C0213079F5B2
:102E800040E050E061E070E0408B518B628B738BCF
:102E9000E801488159816A817B8140835183628343
:102EA000738340A351A362A373A34D915D916D9170
:102EB0007C91139740875187628773878D919D918D
:102EC0000D90BC91A02DB095A095909581959F4FA8
:102ED000AF4FBF4F808F918FA28FB38F30C0223002
:102EE00071F540E050E061E070E040A351A362A3BF
:102EF00073A3E801488159816A817B8140835183B2
:102F000062837383408B518B628B738B4D915D9188
:102F10006D917C91139744835583668377838D915C
:102F20009D910D90BC91A02DB095A0959095819507
:102F30009F4FAF4FBF4F84879587A687B787DF9195
:102F4000CF911F910F910895FC0180E3DF011D9245
:102F50008A95E9F781E082A3828B828308952F927C
:102F60003F924F925F926F927F928F929F92AF9219
:102F7000BF92CF92DF92EF92FF920F931F93CF9366
:102F8000DF93CDB7DEB72A970FB6F894DEBF0FBE3A
:102F9000CDBF4C017A8769871A0100E010E0C101BA
:102FA000800F911F9C838B83D401A00FB11FBA8324
:102FB000A983E12CF12CF8013496F887EF83698519
:102FC0007A856E0D7F1D8B819C810E943A092B01B1
:102FD0003C01A12CB12CC12CD12CC7010C969E8395
:102FE0008D836D817E816A0D7B1DA985BA856A0FEF
:102FF0007B1F8F8198858C0D9D1D820D931D0E94D6
:103000003A09460E571E681E791EB4E0CB0ED11C3D
:10301000ECE0AE0EB11CF8E0CF16D10411F7A98197
:10302000BA814D925D926D927D92BA83A983B4E08C
:10303000EB0EF11CECE0EE16F10409F6045F1F4FF5
:103040000033110509F0ABCFF40109851A850C5D39
:103050001F4F24E0215034962223A9F0D801CD90AF
:10306000DD90ED90FD908D0140A151A162A173A171
:10307000D701C601840F951FA61FB71F80A391A378
:10308000A2A3B3A3E7CF2A960FB6F894DEBF0FBE74
:10309000CDBFDF91CF911F910F91FF90EF90DF9007
:1030A000CF90BF90AF909F908F907F906F905F90E8
:1030B0004F903F902F900895CF92DF92EF92FF9222
:1030C0000F931F93CF93DF93CDB7DEB72C970FB637
:1030D000F894DEBF0FBECDBF8C016B017A018CE08E
:1030E000F801B496DE01119601900D928A95E1F7F0
:1030F0009A01A801BE016F5F7F4F83E00E945707CE
:1031000097012C5F3F4FA801445F5F4FBE016F5F87
:103110007F4F83E00E9457079701285F3F4FA80128
:10312000485E5F4FBE016F5F7F4F83E00E9457078D
:103130008CE0FE013196D60101900D928A95E1F75F
:103140002C960FB6F894DEBF0FBECDBFDF91CF91A6
:103150001F910F91FF90EF90DF90CF9008954F92C5
:103160005F926F927F928F929F92AF92BF92CF9217
:10317000DF92EF92FF920F931F93CF93DF93CDB720
:10318000DEB728970FB6F894DEBF0FBECDBF2C0177
:103190008B017A013A0184E0680E711C5B01E8E062
:1031A000AE0EB11CB301C5010E943A0969837A834E
:1031B0008B839C834701F8E08F0E911C680184E0AB
:1031C000C80ED11CB401C6010E943A096D837E83EA
:1031D0008F839887BE016F5F7F4FCE0105960E9457
:1031E0002509F2016083718382839383B401C8014E
:1031F0000E943A0969837A838B839C83B701C50156
:103200000E943A096D837E838F839887BE016F5F2A
:103210007F4FCE0105960E942509F20164837583D4
:1032200086839783B701C6010E943A0969837A832E
:103230008B839C83B301C8010E943A096D837E830E
:103240008F839887BE016F5F7F4FCE0105960E94E6
:103250002509F201608771878287938728960FB6C8
:10326000F894DEBF0FBECDBFDF91CF911F910F91BC
:10327000FF90EF90DF90CF90BF90AF909F908F9096
:103280007F906F905F904F900895EF92FF920F9311
:103290001F93CF93DF93EC018B01BA01A8010E9429
:1032A000AF18BE0183E00E949B167E018CE0E80E01
:1032B000F11CAE01B801C7010E94AF18B70183E04D
:1032C0000E949B168CE0F801DE01589601900D9249
:1032D0008A95E1F7DF91CF911F910F91FF90EF90C9
:1032E0000895AF92BF92CF92DF92EF92FF920F9329
:1032F0001F93CF93DF93CDB7DEB768970FB6F894DF
:10330000DEBF0FBECDBF8C017B015A016901CE012A
:103310000D960E94AF18BE01635F7F4F83E00E944D
:103320009B16A701BE01635F7F4FCE0101960E94ED
:10333000AF18BE016F5F7F4F83E00E949B168D85A3
:103340009E85AF85B889F80180839183A283B3837A
:1033500089899A89AB89BC8984879587A687B7872D
:103360008D899E89AF89B88D808F918FA28FB38F01
:10337000AE01435F5F4FB60183E00E94D1159B0110
:10338000AC0188279927DC01821B930BA40BB50B9A
:10339000F80184A395A3A6A3B7A389819A81AB81E1
:1033A000BC8184839583A683B7838D819E81AF8101
:1033B000B885808B918BA28BB38B89859A85AB85E1
:1033C000BC85848F958FA68FB78FA501B60183E04A
:1033D0000E94D1159B01AC0188279927DC01821B33
:1033E000930BA40BB50BF80180A791A7A2A7B3A7D5
:1033F000F70180819181A281B381B095A0959095CC
:1034000081959F4FAF4FBF4FF80180879187A2876B
:10341000B387F70184819581A681B781B095A09586
:10342000909581959F4FAF4FBF4FF801848B958B3F
:10343000A68BB78BF70180859185A285B385B09562
:10344000A095909581959F4FAF4FBF4FF80180A3F6
:1034500091A3A2A3B3A3A701B60183E00E94D11553
:10346000F80164A775A786A797A768960FB6F89482
:10347000DEBF0FBECDBFDF91CF911F910F91FF90A7
:10348000EF90DF90CF90BF90AF9008954F925F92F2
:103490006F927F92AF92BF92CF92DF92EF92FF92A4
:1034A0000F931F93CF93DF9300D000D0CDB7DEB73B
:1034B0005C018B01012F1127029506950770872F5C
:1034C00086958F70DB01B17090E000FF1BC0EFE0CC
:1034D000F0E0E81BF90BEE0FFF1FE057FE4F4590A1
:1034E0005490E0E1F0E0E81BF90BEE0FFF1FE0570E
:1034F000FE4F2591349180E092E0AC014A1B5B0BBA
:10350000DA010EC0FC01EE0FFF1FE057FE4F4590A1
:103510005490FC01EE0FFF1FEE56FE4F25913491A3
:10352000612C712CA90160E070E09A01AB012419B3
:103530003509460957090E94D5356B017C0189E0A0
:10354000F594E794D794C7948A95D1F7C40CD51C09
:10355000E61CF71CEE24FF24A7019601C701B60163
:103560000E945535AB01BC019EE075956795579556
:1035700047959A95D1F780E090E0A1E0B0E0841BF8
:10358000950BA60BB70B89839A83AB83BC83CE01C3
:1035900001960E945014CC0CDD1CEE1CFF1C2DEF7C
:1035A000200F2C7F41F4F094E094D094C094C11C7F
:1035B000D11CE11CF11CF501C482D582E682F782A0
:1035C000F501C480D580E680F780C082D182E28296
:1035D000F3820F5F01FB222720F92027322F359538
:1035E0003595232720FD07C09095809570956195AE
:1035F0007F4F8F4F9F4FF50101FF05C06483758397
:103600008683978304C060837183828393830F9042
:103610000F900F900F90DF91CF911F910F91FF901E
:10362000EF90DF90CF90BF90AF907F906F905F90C2
:103630004F900895FF920F931F93CF93DF93CDB7D1
:10364000DEB728970FB6F894DEBF0FBECDBF8C0152
:10365000762FF42E60E0CE0101960E94461A2F2D9F
:10366000AE014B5F5F4FBE016F5F7F4FC8010E948D
:10367000011728960FB6F894DEBF0FBECDBFDF91BD
:10368000CF911F910F91FF90089581BD92BDF89445
:1036900081E08FBB1FBA789480B50895F999FECF69
:1036A00081BD92BD60BDF89484E08FBBF99A789497
:1036B000F999FECF0895AC0110926706E8E6F6E0AE
:1036C00024E0215071F086E090E08150990F88232A
:1036D00031F0342F3170932B56954795F6CF919357
:1036E000F0CF10926B0608958132FCF0813634F4ED
:1036F000E82FEE0FFF0BE05DFD4F0FC08B3734F46A
:10370000E82FEE0FFF0BE051FE4F07C08F3769F037
:10371000E82FEE0FFF0BE450FE4F85919491009738
:1037200021F00E945B1B81E0089580E00895E7E6A8
:10373000F6E034E0315081F02181822F90E0AC013D
:10374000440F551F95958795842B822B9081982B3C
:103750009193822B8083EECFEBE6F6E094E09150DC
:1037600031F0319721818081822B8183F8CF0895B8
:103770001F93CF93DF93C82F83FF04C08FEF9FE782
:103780000E945B1BC0FD0E94971BC4FF04C0809178
:10379000680680936706909166069C3708F04FC0D4
:1037A000809165068A3308F04AC0482F477058E078
:1037B000541BE0E8F0E0E91BF10993E0EE0FFF1F76
:1037C0009A95E1F790E023E0959587952A95E1F7A2
:1037D000E80FF91FE15DFD4FA7E6B6E0D6E01C2F2C
:1037E00012708C2F8470D15051F12D9130E0B901BD
:1037F000042E01C0660F0A94EAF7112329F0C08154
:10380000962F90959C239083882319F090816927A7
:103810006083423090F0052E02C0359527950A94BA
:10382000E2F7112329F06181922F909596239183DD
:10383000882319F09181292721833897D4CFDF91EC
:10384000CF911F91089580911801882359F080919C
:1038500066068C3738F010926606809165068A5F9E
:10386000809365060895EF92FF921F93CF93DF93A5
:103870007C010E94231CC9E1D1E0199111110BC0F8
:10388000809166068C5F80936606DF91CF911F91D1
:10389000FF90EF900895C7010E945B1B812F0E944B
:1038A000B81B81E0CC31D80741F7EACFEF92FF9205
:1038B0000F931F93CF93DF93082F0E94231CC9E11E
:1038C000D1E08CE1E82E81E0F82E1991112359F016
:1038D000802F0E94741B882331F0812F0E94B81B17
:1038E000EC16FD0691F7809166068C5F8093660664
:1038F000DF91CF911F910F91FF90EF900895CF939B
:10390000DF93FC018491EF012196882321F00E942E
:10391000561CFE01F7CFDF91CF9108954F925F9231
:103920006F927F92AF92BF92CF92DF92EF92FF920F
:103930000F931F93CF93DF93CDB7DEB72C970FB6BE
:10394000F894DEBF0FBECDBF6B017C0197FF0BC0AB
:10395000F094E094D094C094C11CD11CE11CF11CE3
:103960008DE20E94561C00E09AE0492E512C612CF9
:10397000712C102FAA24A394B12CAC0EBD1EA00E46
:10398000B11C07FDBA94C701B601A30192010E94C0
:10399000A735605DF501608369017A010F5FC1148D
:1039A000D104E104F10429F71F3F69F0E1E0F0E000
:1039B000EC0FFD1FE10FF11D17FDFA9580810E94AC
:1039C000561C1150F1CF2C960FB6F894DEBF0FBEE7
:1039D000CDBFDF91CF911F910F91FF90EF90DF90BE
:1039E000CF90BF90AF907F906F905F904F90089571
:1039F000FC01909184069F5F923019F090938406A9
:103A000002C010928406409184062CE04203D0014B
:103A10001124A459B94F01900D922A95E1F762E261
:103A20007BE080E090E00C940A32CF93DF93EC01CE
:103A300089858450898768858CE06802B0011124EB
:103A40006C58794FCE010E9480318091830783703A
:103A500029F461E08CE496E00E9499128985881F20
:103A60008827881FDF91CF9108950F931F93CF93DD
:103A7000DF93CDB7DEB728970FB6F894DEBF0FBE41
:103A8000CDBF8C01FC01718560E0CE0101960E94E2
:103A9000461A80915D0690915E0681FF0FC0898174
:103AA0009A81AB81BC81B095A095909581959F4FEF
:103AB000AF4FBF4F89839A83AB83BC8389819A813F
:103AC000AB81BC8124E0880F991FAA1FBB1F2A95D8
:103AD000D1F780932F0190933001A0933101B093DF
:103AE000320180933F0190934001A0934101B09334
:103AF000420180934F0190935001A0935101B093E4
:103B00005201F80120853CE02303F0011124E4591F
:103B1000F94FA3E5B1E001900D923A95E1F72896AF
:103B20000FB6F894DEBF0FBECDBFDF91CF911F91CE
:103B30000F910895CF9320918506822F65E00E9412
:103B40006535C92F2F5F2093850684E690E00E949B
:103B50009226C43011F467E001C066E088E496E084
:103B60000E9499128C2F90E00196880F991F880F60
:103B7000991F80934B06CF910895FC019091850683
:103B8000953038F095509093850681E39BE09383C0
:103B9000828380E008958F929F92AF92BF92CF92DE
:103BA000DF92EF92FF928090890690908A06A09013
:103BB0008B06B0908C06A50194016EE171E78EE052
:103BC0009EE30E9455356B017C010B2C000CC11C3F
:103BD000D11CE11CF11C87EBC81A8AEFD80A86EFCA
:103BE000E80A8EEEF80AC0928906D0928A06E09220
:103BF0008B06F0928C060E941128A701960144279B
:103C00005527DC01BA950E94D535FF90EF90DF90E3
:103C1000CF90BF90AF909F908F900895282FFC0178
:103C20008E2F821B949131969F3FD1F708950F9369
:103C30001F93CF93DF938091A40780FF07C0E0918B
:103C4000860681E0E827E093860605C0E0918D06B0
:103C5000F0918E06E491EF3F09F08CC080918706C9
:103C60009FEF980F90938706811159C00E94CB1D3A
:103C7000A0E0B0E045E0B695A795979587954A9561
:103C8000D1F78F5F8093870640915B0750915C0767
:103C900060915D0770915E074130510591E06907C1
:103CA000710528F1615071093DE07695679557954A
:103CB00047953A95D1F74F3F51056105710529F0B8
:103CC00020F04FEF50E060E070E08A019B01080FA8
:103CD000111D211D311D0F3F11052105310520F05A
:103CE0008FEF8093870603C0480F4093870680912B
:103CF00088069FEF980F90938806811112C00E944A
:103D0000CB1DA0E0B0E026E0B695A79597958795E6
:103D10002A95D1F78F5F80938806E1E003C0E3E046
:103D200001C0E2E0F0E0EE0FFF1FE951FB4FC5914B
:103D3000D491CE010E940E1E182F0E941128DC0182
:103D4000BA95212F30E00E94C6357D5F012F711793
:103D500008F4072F0E94CB1D202F30E0DC010E94C9
:103D6000C635711710F07FEF710FFE01E70FF11DDF
:103D7000E49109C080918D0690918E0601969093F2
:103D80008E0680938D06F0E0EE0FFF1FE55CFA4F84
:103D900085919491909391068093900681E0809311
:103DA0008F06DF91CF911F910F91089541E45FE25B
:103DB00064E973E14093890650938A0660938B0609
:103DC00070938C061092870610928806E82FF0E018
:103DD000EE0FFF1FE951FB4F8591949190938E0652
:103DE00080938D060C94171E80918F06882399F17D
:103DF000815080938F0681112EC080918F06811192
:103E00002AC08091900690919106FC0164916F3FC9
:103E100039F40E94171E80918F068111EECF08950C
:103E2000662351F06F73FFE06F9FB0011124655658
:103E3000754F40E00E940A32809190069091910661
:103E4000FC013396E491E0938F06049690939106DB
:103E500080939006D2CF0895DC011896EC91B0E1E2
:103E6000EB02F0011124EE56F94F8CE0A3E5B1E02E
:103E700001900D928A95E1F70895AF92BF92CF928B
:103E8000DF92EF92FF920F931F93CF93DF93CDB703
:103E9000DEB72C970FB6F894DEBF0FBECDBF7C0106
:103EA0005B0102E916E0D80190E01F962C911F9764
:103EB000242309F09F5F509687E0A235B807A9F741
:103EC000963008F068C090E0F801878581115DC0E8
:103ED000F42FF170CF2E40FF03C064E07BE002C0FE
:103EE00063E17BE0D42E492F80E090E00E940A320B
:103EF000882309F450C0F801D7868CE0F501DE0173
:103F0000119601900D928A95E1F7BE016F5F7F4F88
:103F100083E00E949B1689819A81AB81BC812AE053
:103F2000B595A795979587952A95D1F7F801848738
:103F30008D819E81AF81B8853AE0B595A79597951B
:103F400087953A95D1F7858749855A856B857C8514
:103F5000EAE07595679557954795EA95D1F7CC2096
:103F600019F014160CF44195F80146878CE0F7011E
:103F7000D80101900D928A95E1F7AE014F5F5F4F36
:103F8000B80183E00E94FE1506C09F5F005F1F4FCF
:103F90009C3009F099CF2C960FB6F894DEBF0FBE77
:103FA000CDBFDF91CF911F910F91FF90EF90DF90E8
:103FB000CF90BF90AF9008954F925F926F927F9293
:103FC0008F929F92AF92BF92CF92DF92EF92FF9229
:103FD0000F931F93CF93DF931F92CDB7DEB77C0172
:103FE000DC0118960C91B0E10B02800111240E56F1
:103FF000194FF80167858484208131814281538182
:10400000D58484819581A681B781C68440845184FA
:1040100062847384082C000C9908AA08BB0861FF0D
:1040200032C069E0880C991CAA1CBB1C6A95D1F7A8
:10403000BA01A901480D591D6A1D7B1D408351839A
:10404000628373834D2DDD0C550B660B770B29E0D6
:10405000440F551F661F771F2A95D1F7480F591F28
:104060006A1F7B1F44835583668377838C2DCC0C1A
:10407000990BAA0BBB0B39E0880F991FAA1FBB1F16
:104080003A95D1F732C06BE0880C991CAA1CBB1C76
:104090006A95D1F7BA01A901480D591D6A1D7B1D0A
:1040A000F80140835183628373834D2DDD0C550BE2
:1040B000660B770B2BE0440F551F661F771F2A9561
:1040C000D1F7480F591F6A1F7B1F448355836683AE
:1040D00077838C2DCC0C990BAA0BBB0B3BE0880F84
:1040E000991FAA1FBB1F3A95D1F7480E591E6A1E89
:1040F0007B1E4086518662867386B801685F7F4F5B
:10410000C7010E948031F80180859185A285B38521
:10411000A05ABF4F0197AE45B10598F5F8018081CF
:104120009181A281B38190960197A044B10548F591
:10413000F80184819581A681B78190960197A0446A
:10414000B105F8F4198221E0A80164E0CE010196DE
:104150000E94CA345C01892BB9F41982D8011F96D8
:104160008C9181FF02C062E001C061E022E0A80101
:10417000CE0101960E94CA345C01892B29F480E0AB
:1041800049C0F801178645C0D5011296ED91FC9102
:104190001397949091FE17C0809153079091540704
:1041A000892B89F480915707882351F084E690E0A9
:1041B0000E94922663E088E496E00E94991203C070
:1041C000C5010E94632290FE1AC0F5018185181670
:1041D000B4F4D70119969C91981744F4891B8187F0
:1041E00064E08CE496E00E94991209C0F501118602
:1041F00088EE93E00E949226C8010E94F81C92FE6D
:1042000005C063E08CE496E00E949912D8011F96E5
:104210001C9281E00F90DF91CF911F910F91FF9041
:10422000EF90DF90CF90BF90AF909F908F907F9056
:104230006F905F904F9008950F931F93CF93DF93EC
:10424000CDB7DEB764970FB6F894DEBF0FBECDBF13
:104250008C0180E090E0AFEFBFEFF801808791879D
:10426000A287B38780E091E0A0E0B0E0898B9A8BD1
:10427000AB8BBC8B9E012F5E3F4F43E657E0BE01E8
:10428000675F7F4F82E00E944A0788E0FE0139960F
:10429000DE01119601900D928A95E1F788E0FE010A
:1042A0003196DE01199601900D928A95E1F788E02A
:1042B000FE013996D80101900D928A95E1F7B80177
:1042C00083E00E949B1664960FB6F894DEBF0FBE83
:1042D000CDBFDF91CF911F910F91089588E0E3E664
:1042E000F7E0DF01982F1D929A95E9F7E7E7F7E0ED
:1042F000DF011D928A95E9F780E090E0A8EFBFEF1B
:1043000080879187A287B387109252071092540733
:104310001092530710925A0710925907109258079B
:104320001092550781E080938407109273071092D2
:104330007407109275071092760740E06BE97AE0F7
:1043400080E090E00C940A328091590781111EC0E0
:1043500080912E01982F9670C9F090915A07847021
:1043600091110AC011F081E001C08FEF80935907CD
:1043700084E180935A070895882311F082E001C0F8
:104380008EEF809359078CE28093570708950F931F
:104390001F93CF93DF93CDB7DEB7A8970FB6F894EE
:1043A000DEBF0FBECDBF8E01075E1F4F8CE0F80150
:1043B00011928A95E9F780E090E0A1E0B0E08D8F5E
:1043C0009E8FAF8FB8A38091630790916407A091EF
:1043D0006507B0916607898F9A8FAB8FBC8F68E3B2
:1043E000C8010E94B21480E091E0A0E0B0E08983AF
:1043F0009A83AB83BC83BE016F5F7F4FC8010E946D
:1044000018098CE0E7E7F7E0DE01119601900D92C4
:104410008A95E1F74BE657E0BE016F5F7F4F83E07F
:104420000E9421168CE0FE013196DE011D9601905E
:104430000D928A95E1F7BE01635F7F4F83E00E9492
:104440009B16B80183E00E949B162BE637E0A8017B
:10445000BE01635F7F4F8FE591E00E94711980E09C
:1044600090ECA0E0B0E08DA39EA3AFA3B8A7BE01DF
:104470006B5D7F4F83E891E00E94180980E090EE29
:10448000A0E0B0E08DA39EA3AFA3B8A7BE016B5D73
:104490007F4F87E891E00E941809EFE5F1E080A5E1
:1044A00091A5A2A5B3A5139780A791A7A2A7B3A78B
:1044B000A8960FB6F894DEBF0FBECDBFDF91CF91A7
:1044C0001F910F910895CF93DF932091A40720FDB2
:1044D0001FC026E02093A00720E330E0309354076C
:1044E00020935307FC012185222391F0EC0161E028
:1044F00088E496E00E94991289858150898781110C
:1045000007C081E08093520710925407109253071E
:10451000DF91CF910895EF92FF920F931F93CF9366
:10452000DF93CDB7DEB7A0970FB6F894DEBF0FBE0E
:10453000CDBF7C0180E895E0D70115969C938E93C2
:10454000149780911C018F5F80931C01809152070A
:104550008111EEC08091530790915407009729F084
:10456000019790935407809353078091A40780FD8F
:10457000CCC020912E0122FF1DC03091590780919F
:10458000630790916407A0916507B0916607313089
:1045900011F41E9603C03F3F59F4149680936307AD
:1045A00090936407A0936507B093660711E003C07A
:1045B0001896F4CF10E021FF1CC03091590780916C
:1045C000630790916407A0916507B09166073F3F2C
:1045D00011F41E9705C0313011F4149701C01897DB
:1045E0008093630790936407A0936507B093660771
:1045F00011E023FF12C08091670790916807A09196
:104600006907B0916A0718978093670790936807C6
:10461000A0936907B0936A0711E020FF12C0809150
:10462000670790916807A0916907B0916A0718968B
:104630008093670790936807A0936907B0936A0710
:1046400011E080915A07882319F0815080935A070E
:1046500080912D0184FF06C080915907811102C00D
:104660000E94A42180912C0184FF06C080915907EB
:10467000811102C010925A0780912D0186FF06C059
:1046800083E08093550781E08093560780912E0147
:1046900086FF0CC080915507882351F090915607F2
:1046A000915009F42EC29093560702C010925507FC
:1046B00080915807805E813448F180915307909132
:1046C0005407892B19F580917B0790917C07A09165
:1046D0007D07B0917E0781309048A105B105B4F403
:1046E000C7010E946322D70119968C91882371F02B
:1046F00080E090E0A0E0B1E08093670790936807C6
:10470000A0936907B0936A0701C010E080E090EEC3
:10471000A0E0B0E089839A83AB83BC839E012F5FC6
:104720003F4F43E657E0BA0182E00E944A077FC04C
:104730001092590740917B0750917C0760917D074B
:1047400070917E078130D9F5809167079091680755
:10475000A0916907B0916A071297809367079093B9
:104760006807A0936907B0936A0714161506160622
:1047700017068CF080E090E0A0E4B0E0809367073B
:1047800090936807A0936907B0936A0764E088E490
:1047900096E00E949912809153079091540721E06E
:1047A000803F910508F020E020938407803F910529
:1047B000E8F187E797E00E94F81C81E000C2809151
:1047C000770790917807A0917907B0917A07B09513
:1047D000A095909581959F4FAF4FBF4FF4E0B59551
:1047E000A79597958795FA95D1F78093630790934E
:1047F0006407A0936507B093660780E090E0A8E0A7
:10480000B0E0841B950BA60BB70B14E0B595A795EC
:10481000979587951A95D1F78093670790936807C6
:10482000A0936907B0936A0710E001C011E080917E
:104830005907882309F44DC080915707882369F0F0
:10484000815080935707811108C0109259078091B9
:104850002E0184FF1AC00E94A421809159078E3F27
:1048600049F49091570790310CF09FE080915807E0
:10487000891B44C0823051F48091570780310CF07D
:104880008FE090915807890F39C080E090912E01F8
:1048900094FD03C01092590733C0813061F48091B8
:1048A0005807B3E08B02C001112495958795959523
:1048B0008795805F23C08F3F19F580915807E3E00B
:1048C0008E02C00111249595879595958795805105
:1048D00015C080915807882399F080FF05C087FF95
:1048E00003C08F5F8093580780915807F3E08F02D1
:1048F000C0011124959587959595879580935807C4
:10490000111109C020E030E140E050E063E677E0BB
:1049100082E00E94E71480E091E0A0E0B0E08D8F9B
:104920009E8FAF8FB8A39E01235E3F4F43E657E0B3
:10493000BE016F5F7F4F82E00E944A0788E0FE0160
:104940003196DE011D9601900D928A95E1F788E07F
:10495000FE013D96DE01559601900D928A95E1F794
:1049600088E0FE017596DE01119601900D928A9500
:10497000E1F7AE014F5F5F4F67E777E082E00E94AB
:10498000FE158091A40780FF29C0809152078111F4
:1049900025C0809183078093580780E090E0A0EFC6
:1049A000BFEF8093770790937807A0937907B09330
:1049B0007A0780E090E0A0E1B0E080937B079093DD
:1049C0007C07A0937D07B0937E078CE0E7E7F7E0D4
:1049D000ABE6B7E001900D928A95E1F760E187E7D9
:1049E00097E00E94B21460E18BE797E00E94B21456
:1049F00080917B0790917C07A0917D07B0917E0705
:104A0000B7FF08C010927B0710927C0710927D07B9
:104A100010927E078CE0E7E7F7E0DE011196019047
:104A20000D928A95E1F78D819E81AF81B88590586E
:104A3000AF4FBF4F8D839E83AF83B88780E090E2F6
:104A4000A0E0B0E08D8F9E8FAF8FB8A38E01035E84
:104A50001F4F9E012F5F3F4F4BE657E0BA0183E0A7
:104A60000E945615109273071092740710927507E2
:104A70001092760780915207882309F45AC081303A
:104A800009F09CC080915307909154078937910594
:104A900010F088E790E0A0E0B0E08C019D014AE0D2
:104AA000000F111F221F331F4A95D1F740916B074A
:104AB00050916C0760916D0770916E07401B510B10
:104AC000620B730B40936B0750936C0760936D07F9
:104AD00070936E0754E0880F991FAA1FBB1F5A9549
:104AE000D1F7B095A095909581959F4FAF4FBF4F4F
:104AF0008093730790937407A0937507B09376071C
:104B00005DC09CE090935607815080935507CE017D
:104B100001960E941C2141E0BE016F5F7F4F87E735
:104B200097E00E943D1F60E088E496E00E949912A1
:104B3000BFCD19828091530790915407892B09F0BA
:104B40003DC021E047E757E065EBCE0101960E94AA
:104B5000CA348C01009791F1DC011296ED91FC9121
:104B60001397E491E7FF05C0FC0111860E949A1D8E
:104B700025C0E5FF20C0D70119968C9119978E5F4B
:104B80008A301CF419968C9303C08AE0F701818760
:104B900062E088E496E00E94991280ED97E00E941E
:104BA000922680E390E09093540780935307C801C6
:104BB0000E94A03103C0C7010E94632280E0A0963A
:104BC0000FB6F894DEBF0FBECDBFDF91CF911F911E
:104BD0000F91FF90EF9008950F931F93CF93DF9362
:104BE000CDB7DEB7C857D1090FB6F894DEBF0FBEF8
:104BF000CDBF8E0103591F4F8CE0F80111928A95A9
:104C0000E9F780E090E0A1E0B0E0F80184839583CB
:104C1000A683B7838091590781111AC080916307D9
:104C200090916407A0916507B09166078083918396
:104C3000A283B38380E092E0A0E0B0E089839A830E
:104C4000AB83BC83BE016F5F7F4FC8010E94180910
:104C5000CE018F599F4F0E941C21A801BE016F59A0
:104C60007F4F8FE291E00E94451942E06091580722
:104C7000CE01C1960E941A1B80E3FE01F196DE016F
:104C8000119601900D928A95E1F7AE014F5F5F4F4B
:104C90006FE271E0CE01C1960E94AF1780E3FE0182
:104CA000F196AFE2B1E001900D928A95E1F780E0D4
:104CB00090E0A2E0B0E089839A83AB83BC83BE011D
:104CC0006F5F7F4F8FE291E00E94FB168CE0E7E779
:104CD000F7E0A3E5B1E001900D928A95E1F7C8589D
:104CE000DF4F0FB6F894DEBF0FBECDBFDF91CF917F
:104CF0001F910F9108950F931F93FB01DC014D91BC
:104D00005D916D917C9180819181A281B3818A01B5
:104D10009B01080F191F2A1F3B1FC901B8011F91D2
:104D20000F910895EBE5F7E0408151816281738135
:104D3000480F591F611D711D408351836283738326
:104D400021E02093A3079093A2078093A1070895E1
:104D5000AF92BF92CF92DF92EF92FF920F931F9389
:104D6000CF93DF9300D000D0CDB7DEB76C018C01BC
:104D70008BE5E82E87E0F82ECE0101965C01C80194
:104D80000E94451BF7018483C80104960E94451BBD
:104D9000F70181937F01C80108960E94451BF50128
:104DA00081935F010F5F1F4FFFE5EF16F7E0FF06EE
:104DB00031F7C6010C960E94451B8270816080937A
:104DC000A40749815A816B817C818FE548278AE855
:104DD000582781EA682785EF782780915B079091B3
:104DE0005C07A0915D07B0915E0780959095A095B6
:104DF000B09500915F071091600720916107309195
:104E0000620780179107A207B30729F448175907CB
:104E10006A077B0759F010925F07109260071092A3
:104E200061071092620783E08093A40710925B07EA
:104E300010925C0710925D0710925E070F900F9022
:104E40000F900F90DF91CF911F910F91FF90EF90F6
:104E5000DF90CF90BF90AF9008958F929F92AF92C6
:104E6000BF92CF92DF92EF92FF920F931F93CF9357
:104E7000DF9300D000D0CDB7DEB76C0180915F0723
:104E800090916007A0916107B09162072FE582279A
:104E90002AE8922721EAA22725EFB22789839A835D
:104EA000AB83BC8386018FE5E82E87E0F82ECE0128
:104EB00001965C014701F70161917F01C8010E94E1
:104EC0004E1BF40160816095C80104960E944E1B40
:104ED000F50161915F01C80108960E944E1B0F5FAA
:104EE0001F4FF3E6EF16F7E0FF0621F76091A407E6
:104EF000C6010C960F900F900F900F90DF91CF91FD
:104F00001F910F91FF90EF90DF90CF90BF90AF90E7
:104F10009F908F900C944E1BEF92FF920F931F93D4
:104F2000CF93DF931BE6F12E28E138E0AFE8B2E043
:104F3000FA94FF2009F46EC0F901649131967491DE
:104F40002D5F3F4F31965491F901E49031960491D1
:104F5000319614913196E4916E29462F4E2BF9012A
:104F600034969491E72FE02B9E2BF901359684918E
:104F7000E52FE12B8E2B642F70E0C92FD0E0FB01D1
:104F8000EE0FFF1F759567956E2B642BAE0156953E
:104F9000542F442757954795F62FF42B682F70E030
:104FA000AE01440F551FD595C795C42BC92BAB0136
:104FB0005695542F4427579547954C2BEF2FEE1FAE
:104FC000EE27EE1F4E2BF0959C91F923EF2AEC92E1
:104FD000E42FE09511969C911197E9230E2B1196E1
:104FE0000C931197FB01EE0FFF1F759567956E2BC4
:104FF000E62FE82B842F881F8827881F8E2B80950B
:105000001296EC9112978E23182B12961C931297DE
:1050100018968ECFDF91CF911F910F91FF90EF9057
:10502000089580915B0790915C07A0915D07B09116
:105030005E0729E0B695A795979587952A95D1F7AC
:10504000813021E09207A105B10520F080E091E0D8
:10505000A0E0B0E0939508950E94743280E591E05D
:10506000E5EAF7E0DF019C011D9221503040E1F7B5
:1050700080ECE2E9F6E0DF011D928A95E9F70E94F3
:105080006E211092850680E00C94D61EE0E1F8E0D7
:10509000E491E0938707E1E1F8E0E491E093880789
:1050A000E2E1F8E0E491E0938907E3E1F8E0E491DC
:1050B000E0938A07A3E9B7E080E090E0FC01EC5EB2
:1050C000F74FE491ED93019684309105B9F7089577
:1050D0002F923F924F925F926F927F928F929F9208
:1050E000AF92BF92CF92DF92EF92FF920F931F93F6
:1050F000CF93DF9300D01F92CDB7DEB740915D060E
:1051000050915E06242E082E000C990B062E000CE2
:10511000770B681B790B660F771F062E000C770B39
:10512000982F88279B0135952795820F931F9A8387
:105130008983A0E83A2E340E8FE292E0B8E0AB2EDD
:105140001BE0412E55245A940CE0902E231409F4B0
:1051500077C0EA812E2F0E2E000C330B43E03595DD
:1051600027954A95E1F7522F27FF05C0422F419519
:1051700028E050E00CC0233034F02D3034F4442DBE
:10518000421B242F03C028E001C020E040E03E2F56
:105190003770BA2CB21ABB82F42E241BFC0141508A
:1051A00010F05192FCCF8F0D911D2394022D0170B0
:1051B00010E0909EF001919EF00D1124E957F84FF8
:1051C000E50FF11D57FDFA953323E9F08A2C831A78
:1051D00041917C01722E7A945FEF7516C1F0619057
:1051E00050E0032E02C0559547950A94E2F7C62C6D
:1051F000082C01C0CC0C0A94EAF74C0DD7014D9352
:105200007D01462DE8CFAC01322F315020F4820FC2
:10521000911DFC0105C0F190DA01FD92AD01F5CFC1
:10522000BB81B150BB83BF3F11F01192F9CF8B0D01
:10523000911D29813A81260F371F3A83298386CF12
:105240000F900F900F90DF91CF911F910F91FF90D2
:10525000EF90DF90CF90BF90AF909F908F907F9016
:105260006F905F904F903F902F9008951092660638
:105270008EE18093650684EC99E00E947F1C0E9479
:105280000212F8942F986DE770E080E090E00E94A1
:10529000090987E797E79093010880930008A8958C
:1052A00088E18093600088E080936000FFCF8AEF00
:1052B000809326098FEA8093270985E58093280942
:1052C00080E190E00E94A8260E94C8070E94E8079B
:1052D0008091A40781FD03C080E090E002C080E8D7
:1052E0009EE30E94081480912E018A3561F4109289
:1052F0005F0710926007109261071092620780E1C9
:1053000090E00E942D270E9400120E942C2880917C
:105310005F06809383070E94462880912E01883083
:1053200011F40E9436291BBC089562E08CE496E0DB
:105330000E94991284E190E0A0E0B0E080935B07C6
:1053400090935C07A0935D07B0935E0710922D01C8
:105350008091A40785608093A407089510925B074D
:1053600010925C0710925D0710925E0710922D015B
:105370000E942C288091A4078A7F8093A407089517
:105380002F923F924F925F926F927F928F929F9255
:10539000AF92BF92CF92DF92EF92FF920F931F9343
:1053A000CF93DF93CDB7DEB7C254D1090FB6F894CF
:1053B000DEBF0FBECDBFEE24E394F12C80915F06DB
:1053C00090918307981709F4D4C10E94E80780914F
:1053D000A40780FF49C082FD5FC080912D0183FF3B
:1053E00005C090919F07915090939F0780FF05C043
:1053F00090919F079F5F90939F07897029F060E0CD
:105400008CE496E00E94991280919F0781708093AE
:105410009F0790912D01907509F43EC09701082EC9
:1054200001C0220F0A94EAF79091A407292720933C
:10543000A407811103C022FF0E94952980919F0734
:10544000813051F58091A40781FF03C080E89EE37D
:1054500002C080E090E00E9408146091A4078CE1F3
:1054600090E00E944E1B18C0809183078F3AA1F4F0
:10547000F89490918307E92FF0E0EF52F74F80E521
:105480002491222331F0880F811D2491820F3196BF
:10549000F7CF891301C07894209152072223C9F1D4
:1054A00080915307909154070196909354078093ED
:1054B0005307213009F044C08134914008F440C0C2
:1054C0008091A40781608093A40780915B079091ED
:1054D0005C07A0915D07B0915E0740915F07509116
:1054E00060076091610770916207481759076A0762
:1054F0007B0760F480935F0790936007A093610738
:10550000B093620780E190E00E942D270E942C2832
:1055100017C08091A40780FD13C080915B07909114
:105520005C07A0915D07B0915E070196A11DB11DBA
:1055300080935B0790935C07A0935D07B0935E0731
:105540008091A007833018F081508093A00780914C
:105550008407882349F10E94112820918507309102
:105560008607820F931F9093860780938507BC015F
:1055700046E0769567954A95E1F7A90176E056955C
:1055800047957A95E1F7B62EB41A192F131B1123FC
:1055900021F00E94F41E1150FACF80918F068111E4
:1055A00004C00E94D61E01C0B12C8091A30788239D
:1055B00051F090E008968F3F910519F014F080E0CB
:1055C00090E08093A307A0902509AA94CB2CD12C1E
:1055D0001FEFA11609F4C7C0EA2DF0E0EE0FFF1F80
:1055E000EB50F74F00811181D80114968D919C9159
:1055F00015978C0D9D1D15969C938E9314976B2D6E
:10560000C8010E942733882379F0BE01635F7F4F72
:10561000C8010E94C4348D899E89AF89B88D0197D5
:10562000AE4FBF4F4CF01EC0D80114968D919C9187
:10563000159781309640B4F4D8011296ED91FC9103
:1056400013973B96259134912115310531F0C8010E
:10565000F9010995882359F005C0D80119968C9154
:10566000811105C0C8010E94A031AA94B1CFF801F0
:1056700083858823D1F39091A40790FDF6CF92857E
:105680002FEF290F22879111F0CF0280F381E02DB7
:105690003896E491D8011A96EC931A9781501B968C
:1056A0008C93BE01675E7F4FC8010E94C4348CE0BA
:1056B000E7E7F7E0DE01119601900D928A95E1F798
:1056C000AE01475E5F4FBE016F5F7F4F83E00E9478
:1056D00021168CE0FE013196DE011D9601900D929F
:1056E0008A95E1F7BE01635F7F4F83E00E949B16BE
:1056F0008D859E85AF85B88912E0B595A79597955C
:1057000087951A95D1F78D879E87AF87B88B898942
:105710009A89AB89BC8902E0B595A795979587953D
:105720000A95D1F7898B9A8BAB8BBC8B8D899E891F
:10573000AF89B88D22E0B595A795979587952A955D
:10574000D1F78D8B9E8BAF8BB88F42E0BE01635F2C
:105750007F4FCE0149960E943D1F65E08CE496E0A4
:105760000E94991282CF809183078F5F8093830775
:1057700025CE0E94C72188E0EBE8F7E0DF01E82EA4
:105780001D92EA94E9F7E7E9F7E0DF011D928A95B7
:10579000E9F780E090E0A0EABFEF898F9A8FAB8FA6
:1057A000BC8FBE01675E7F4F8BE791E00E943A0994
:1057B0006D877E878F87988B4E01BDE08B0E911C85
:1057C000B40187E891E00E947B266B017C01FF0C0D
:1057D000CC08DC2C76019B01AC016C2D7C2D8C2D32
:1057E0009C2D00E10E94B736A12CB12CE0EACE2E10
:1057F000DD24DA94EE24EA94FF24FA940FEF1FEFED
:105800000E94E23529AF3AAF4BAF5CAFF6E03F2ED6
:10581000ACE02A2E3A94EFEF3E1609F4A5C0209191
:105820008507309186073F73832D90E0A0E0B0E0BC
:105830001EE0880F991FAA1FBB1F1A95D1F7820F70
:10584000931FA11DB11D06E0880F991FAA1FBB1F42
:105850000A95D1F7A056B109898F9A8FAB8FBC8F6B
:10586000BE01675E7F4F8BE791E00E943A096D872A
:105870007E878F87988BB40187E891E00E947B2612
:10588000498C5A8C6B8C7C8C4114510461047104DA
:1058900009F26B017C01FF0CCC08DC2C76019B012A
:1058A000AC016C2D7C2D8C2D9C2D00E10E94B73617
:1058B00083017201110FEE08FE2C87012196ECAED8
:1058C000FDAE0EAF1FAF219752016301EDACFE2C70
:1058D0000E2D1E2D0E94E23559016A01D601C50127
:1058E00029AD3AAD4BAD5CAD821B930BA40BB50B50
:1058F000AC01BD01FAE07595679557954795FA9506
:10590000D1F757FD87CF5A0130E2A30EB11C40E614
:10591000A416B1040CF07ECF532D517022965FAFC8
:10592000229723961FAE2397C50123E0959587956F
:105930002A95E1F72396AEADBFAD23972A9EF001DD
:105940002B9EF00D1124E957F84FE80FF91FB7E02F
:10595000AB22BB2481E090E001C0880FAA94EAF753
:105960009081892B808356CF80E090E0A0E6B0E064
:10597000898F9A8FAB8FBC8F1D8E1E8E1F8E18A2A3
:1059800080E090E0A0EABFEF89A39AA3ABA3BCA3F9
:105990008D879E87AF87B88B198A1A8A1B8A1C8AC3
:1059A0008D8B9E8BAF8BB88FAE01475E5F4FBA0178
:1059B0008FE591E00E945C18A401B4018FE591E0AD
:1059C0000E945C1889A19AA1ABA1BCA1AC01BD0148
:1059D000770F440B542FBA015C016D01E42EF42EB5
:1059E000042F142F20E030E040E050E061E070E050
:1059F00080E090E00E94E2352DA33EA34FA358A77C
:105A0000BE016B5D7F4FCE0149960E941809BE0111
:105A10006B5D7F4FCE014D960E9418098D899E893E
:105A2000AF89B88DAC01BD01770F440B542FBA017B
:105A30005C016D01E42EF42E042F142F20E030E0E1
:105A400040E050E061E070E080E090E00E94E235EC
:105A50002DA33EA34FA358A7BE016B5D7F4FC4018A
:105A60000E941809BE016B5D7F4FCE0141960E94D6
:105A70001809BE01675E7F4FC4010E9425092B01F2
:105A80003C01BE01635E7F4FCE0141960E94250915
:105A90006DAB7EAB8FAB98AF4114510461047104C0
:105AA00029F16B017C01FF0CCC08DC2C76019B01F9
:105AB000AC016C2D7C2D8C2D9C2D00E10E94B73605
:105AC00083017201110FEE08FE2C8701E9AEFAAED8
:105AD0000BAF1CAF52016301E9ACFE2C0E2D1E2D45
:105AE0000E94E2352DAB3EAB4FAB58AF80E090E06B
:105AF000AFEFBFEF89AB9AABABABBCABBE01675EA0
:105B00007F4FCE01C1960E9425096DA37EA38FA36E
:105B100098A7BE016B5C7F4FCE0185960E943A0923
:105B20000D8D1E8D2F8D38A1DC01CB01800F911FB3
:105B3000A21FB31F8D8F9E8FAF8FB8A380E090E020
:105B4000A1E0B0E089AB9AABABABBCABB401CE018A
:105B5000C1960E9425096DA37EA38FA398A7BE01BD
:105B60006B5C7F4FCE0185960E943A0909891A899C
:105B70002B893C89DC01CB01800F911FA21FB31F31
:105B8000898B9A8BAB8BBC8BB095A09590958195AA
:105B90009F4FAF4FBF4FBC01CD015AE09595879500
:105BA000779567955A95D1F70D8D1E8D2F8D38A15C
:105BB00030952095109501951F4F2F4F3F4F7AE05C
:105BC00035952795179507957A95D1F7802F0E94DF
:105BD000682880912E01893041F480915F069BB541
:105BE000891B833828F00E94362980915F068BBD7F
:105BF00080E090E0AEEFBFEF809314019093150129
:105C0000A0931601B093170180E090E0A0EABFEFE7
:105C10008093100190931101A0931201B09313018E
:105C200080E090E0A0E4B0E080936106909362068B
:105C3000A0936306B09364060E94FF098091250932
:105C4000882309F457C1F0902509EFEFEF0DF0E03C
:105C5000EE0FFF1FEB50F74F80819181DC0116960C
:105C60006D917C911797A4010E943A344D885E880B
:105C70006F88788CFA94FA94E12CBFEFFB1609F444
:105C80004BC00F2D10E06801CC0CDD1CF601EB5071
:105C9000F74F80819181FC016681778161157105E3
:105CA00021F0A4010E943A3414C084819581092E08
:105CB000000CAA0BBB0B9650A109B1092CE0880F70
:105CC000991FAA1FBB1F2A95D1F78D8B9E8BAF8B77
:105CD000B88F8D899E89AF89B88D481659066A0696
:105CE0007B0624F0FA942C013D01C7CF000F111F51
:105CF000F801E950F74F80819181D601AB50B74F41
:105D00002D913C911197318320838D939C93D301E6
:105D1000C201EE24E394E6CFE11095CFF12C7CE0B4
:105D2000772E212C312C2101439480912509F816DE
:105D300008F0E0C00F2D10E0000F111FF801EB502C
:105D4000F74F80819181FC0122813381F9013D96D9
:105D5000A590B490F9013A96E4903997C590D49003
:105D6000BE016B5D7F4F0E947E32F6013196E49159
:105D7000EF70D1F040918307440F440F2E2F30E095
:105D80002F5F3F4F429FC001439F900D112490937E
:105D9000150221E0290FE21718F02093140202C027
:105DA0001092140280931302EE2009F461C0AE0138
:105DB000475E5F4F63E571E0F801EB50F74F80817C
:105DC00091810E949434D401E72D1D92EA95E9F760
:105DD000298A3A8A4B8A5C8A898D9A8DAB8DBC8DD3
:105DE00052E0B595A795979587955A95D1F78D87E8
:105DF0009E87AF87B88BA401BE01675E7F4F8FE29D
:105E000091E00E9445198DA19EA1AFA1B8A5009770
:105E1000A140B10589F489A59AA5ABA5BCA50097B9
:105E2000A140B10549F48DA59EA5AFA5B8A90097DD
:105E3000A140B10509F44DC09E012B5D3F4F4FE2DB
:105E400051E0BA0183E00E944A079E01275D3F4F5F
:105E50004BE351E0BA0183E00E944A079E01235DB3
:105E60003F4F47E451E0BA0183E00E944A0731C046
:105E70008FE291E00E94A4178DA19EA1AFA1B8A5C9
:105E800080932F0190933001A0933101B0933201A0
:105E900089A59AA5ABA5BCA580933F01909340012D
:105EA000A0934101B09342018DA59EA5AFA5B8A9CD
:105EB00080934F0190935001A0935101B0935201F0
:105EC00063E571E0F801EB50F74F808191810E940A
:105ED000C434A114B10439F0F801EB50F74F8081BC
:105EE0009181F5010995C6010E94BA0F0E94F80937
:105EF000F3941BCF8091A40780FD44C012E010935F
:105F0000660681E08093650660915B0770915C078F
:105F100080915D0790915E070E948E1C8091A3077F
:105F2000882381F120915D0630915E0620FF06C036
:105F300097E09093190110931A0106C093E0909393
:105F4000190194E090931A0190E0805C91098931E5
:105F5000910514F088E190E022E02093660697FF17
:105F600002C080E090E090E2981B909365068BE27F
:105F70000E94561C6091A1077091A20780E090E0FA
:105F80000E948E1C8091A007882371F0815080931D
:105F9000A00761E070E0882319F08FE098E002C06C
:105FA0008EE098E00E948D088091A40780FF9EC03B
:105FB0000E948C2783E08093190184E080931A016A
:105FC00083E68093660684E1809365068BED99E015
:105FD0000E947F1C88E08093660683E380936506B9
:105FE00080E899E00E947F1C89E18093660689E33E
:105FF000809365068CE699E00E947F1C8BE5E82E75
:1060000087E0F82E98E1C92E00E010E027E0B22EDC
:1060100032E0A32E4CE2942ED02E8091A40782FF72
:1060200021C080915B0790915C07A0915D07B091C2
:106030005E0780FF05C0B0921901A0921A0107C047
:106040000097A105B10519F40E94AE2996C00197E9
:10605000A109B10980935B0790935C07A0935D074A
:10606000B0935E0790926606C092650680919F0786
:106070008D1102C08EE301C080E20E94561CC70150
:106080008B5597402091A40730E0002E02C0359533
:1060900027950A94E2F720FF03C0E2E0F0E002C097
:1060A000E0E0F0E0E80FF91FE45AF64F8591949193
:1060B0000E947F1CDA94DA94D7FC08C0F701389765
:1060C00060817181828193810E948E1C8091A407DE
:1060D00082FD53C00F5F1F4FF4E0EF0EF11C26E06E
:1060E000C20E0430110509F097CF47C08091830795
:1060F00086958695869586704091770750917807AA
:106100006091790770917A074115510531EF630766
:106110003FEF73072CF48E5F809366068EE30AC010
:10612000413051056F40710554F09BE7981B9093E7
:1061300066068CE39AE0909365060E94561C809157
:10614000530790915407892B09F45BC08091520743
:10615000811157C080915D0690915E0680FD56C00A
:1061600050C000FF04C08FE190E00E94331C83E028
:106170008093190184E080931A010E940212809199
:106180005D0690915E06019690935E0680935D0693
:10619000809126098A3F41F4809127098F3A21F4A2
:1061A00080912809853589F061E070E08FE098E002
:1061B0000E948D080E94AF1261E070E08EE098E0CE
:1061C0000E948D080E94AF12EFCF0E94AF12CE5BEB
:1061D000DF4F0FB6F894DEBF0FBECDBFDF91CF917A
:1061E0001F910F91FF90EF90DF90CF90BF90AF90F5
:1061F0009F908F907F906F905F904F903F902F90E7
:10620000089583E08093190184E004C087E08093BF
:10621000190182E080931A010091AE0782E0809319
:10622000660688E38093650683E50E94561C80918C
:106230005207813009F4A1CF102F1695112309F4CC
:1062400090CF8FE19CE70E94331C1150F7CFCF9382
:10625000DF93CDB7DEB72C970FB6F894DEBF0FBE35
:10626000CDBF80915D0690915E06782F7295707F0C
:1062700060E0CE0101960E94461A89819A81AB8125
:10628000BC8124E0880F991FAA1FBB1F2A95D1F754
:1062900089839A83AB83BC83BE016B5F7F4F8FE2A0
:1062A00091E00E941809BE016F5F7F4F87E391E084
:1062B0000E94180989819A81AB81BC81B095A09513
:1062C000909581959F4FAF4FBF4F89879A87AB8736
:1062D000BC87BE01675F7F4F87E491E00E94180989
:1062E000BE016B5F7F4F8BE491E00E9418092C96F2
:1062F0000FB6F894DEBF0FBECDBFDF91CF910895EA
:10630000CF93DF93EC01FB0180819181A281B38166
:10631000BC01CD01805A9F4F20E030E140E050E0C9
:106320000E94A7352130F6E03F071CF43D832C8303
:1063300004C080E096E09D838C83DF91CF91089527
:10634000DC0115961C921E92149720912509E5EF09
:10635000F8E090E09217F9F041915191A417B50738
:10636000C1F48FEF820F809325099817A0F4292F8D
:1063700030E0F901EE0FFF1FE950F74F40815181E6
:10638000220F331FF901EB50F74F518340839F5F7A
:10639000ECCF9F5FDFCF0895CF93DF93EC01909117
:1063A00025099831A1F1A5EFB8E060E0691721F166
:1063B0002D913D914C815D81F90124813581241716
:1063C000350714F0292F02C06F5FF0CF8FEF820FD7
:1063D000621790F4282F30E0D901AA0FBB1FAB50F1
:1063E000B74F4D915C91220F331FD901A950B74F80
:1063F0004D935C93282FEACF9F5F90932509E62F5A
:10640000F0E0EE0FFF1FEB50F74FD183C083DF9119
:10641000CF910895E5EAF7E0A0E024813581232BB0
:1064200009F05BC02EE0A29FD0011124AB55B84FFC
:1064300021E030E015963C932E93149717961C920A
:106440001E92169711969C938E9313967C936E933F
:10645000129718964C931897FB013696E49119966B
:10646000EC931997FB013796E4911A96EC931A97DF
:10647000FB01399664911B966C931B9740917707AB
:10648000509178076091790770917A07505E6F4F4D
:106490007F4F8EE075956795579547958A95D1F70B
:1064A0001C964C931C9740917B0750917C07609100
:1064B0007D0770917E07505E6F4F7F4F9EE0759510
:1064C0006795579547959A95D1F71D964C931D97CB
:1064D000CD010E94CC3181E00895AF5F3E96A83196
:1064E00009F09BCF80E008951092250980E3E5EF45
:1064F000F8E0DF011D928A95E9F70895CF93DF93C5
:10650000EB01FC0182819381FC013396E4914E2FD3
:1065100050E060E070E02EE0440F551F661F771FCB
:106520002A95D1F7488359836A837B83FC0134968B
:10653000E4914E2F50E060E070E03EE0440F551FC4
:10654000661F771F3A95D1F74C835D836E837F83F7
:10655000FC013596E4918E2F90E0A0E0B0E04EE093
:10656000880F991FAA1FBB1F4A95D1F78887998763
:10657000AA87BB87DF91CF9108950F931F93CF9385
:10658000DF93EB01FC014491042E000C550B660BCC
:10659000770BBA0155274427088119812A813B814D
:1065A000400F511F621F731F488359836A837B8387
:1065B0003196E4914E2FEE0F550B660B770BBA0117
:1065C000552744270C811D812E813F81400F511F8B
:1065D000621F731F4C835D836E837F83FC01329641
:1065E000E4918E2FEE0F990BAA0BBB0BDC019927C0
:1065F0008827488559856A857B85840F951FA61F46
:10660000B71F88879987AA87BB87DF91CF911F9192
:106610000F910895DC011296ED91FC9113973A9633
:10662000E491EE2389F09FEF9E0FED91FC91E491B0
:10663000E6FBEE27E0F9E90FF0E0EE0FFF1FEA5E60
:10664000F34F85919491089580E090E008951F9311
:10665000CF93DF93EC01162F0E940A33009771F05D
:10666000FC01319684912E813F81A901819F400DCB
:10667000511D11245F834E8381E001C080E0DF91D2
:10668000CF911F9108952F923F924F925F926F92F8
:106690007F928F929F92AF92BF92CF92DF92EF92B2
:1066A000FF920F931F93CF93DF93CDB7DEB7A497DD
:1066B0000FB6F894DEBF0FBECDBF6C013B012A01BF
:1066C0000E940A33009709F4BCC0FC013490272DC6
:1066D000371410F0262C03C0232D22242A94F6E030
:1066E0002F9F800D911D11248C010E5F1F4FCE0135
:1066F00001967C0184E2D7011D928A95E9F7570142
:106700004801B9E08B0E911CB501C8010E94BD3251
:106710000D5F1F4FECE0AE0EB11C08151905A1F777
:10672000A22CB12C85019E01235F3F4FA701B70129
:1067300083E00E94AD159E01275E3F4FAE01435F8F
:106740005F4FBA0183E00E94AD159E01235F3F4F6A
:10675000A701B70183E00E94AD15D6011296ED9115
:10676000FC911397E491E6FF52C0F6014485042E94
:10677000000C550B660B770B8EE0440F551F661F00
:10678000771F8A95D1F78585082E000C990BAA0BE7
:10679000BB0B2EE0880F991FAA1FBB1F2A95D1F7AC
:1067A00009851A852B853C850D8B1E8B2F8B388F89
:1067B000F2010081118122813381401B510B620B58
:1067C000730B4D875E876F87788B44815581668117
:1067D0007781841B950BA60BB70B898B9A8BAB8BA0
:1067E000BC8B632D70E0962F88278615970524F0C3
:1067F000C3010E94713502C060E071E08B019E010F
:10680000235F3F4FA701B70183E00E94AD15D6017A
:10681000ED91FC91E491E7FF0FC089819A81AB81F2
:10682000BC81B095A095909581959F4FAF4FBF4F7C
:1068300089839A83AB83BC83A701B20183E00E9462
:10684000FE15A4960FB6F894DEBF0FBECDBFDF9144
:10685000CF911F910F91FF90EF90DF90CF90BF905D
:10686000AF909F908F907F906F905F904F903F90F0
:106870002F900895CF92DF92EF92FF920F931F9384
:10688000DA01FC01008111810115110511F1F801F6
:106890003296E491CE2EEE0FDD08EE08FF08760169
:1068A000DD24CC241496CD92DD92ED92FC921797C4
:1068B000F8013196E4910E2FEE0F110B220B330BE2
:1068C0009801112700270D931D932D933C93139747
:1068D0000BC01D921D921D921C92139714961D922F
:1068E0001D921D921C921797FC0104811581012EA7
:1068F000000C220B330B1650210931094CE0000F1C
:10690000111F221F331F4A95D1F718960D931D931F
:106910002D933C931B97AD011F910F91FF90EF902A
:10692000DF90CF900C944333EF92FF920F931F931D
:10693000CF93DF938C017B01EA01FC0166817781B3
:10694000A7010E943A34F80166817781605E7F4F2B
:10695000AE01C8010E943A3488859985AA85BB8515
:10696000119688879987AA87BB87A701BE0183E014
:106970000E942116BE0183E0DF91CF911F910F91FC
:10698000FF90EF900C949B16AB01FC016681778120
:106990000C943A34AF92BF92CF92DF92EF92FF9273
:1069A0000F931F93CF93DF93CDB7DEB76C970FB6DE
:1069B000F894DEBF0FBECDBF6C01062F5A01DC017B
:1069C0001C91822F90E0A0E0B0E02FE0880F991F8B
:1069D000AA1FBB1F2A95D1F7898F9A8FAB8FBC8FC7
:1069E00080912509181708F04BC0E12FF0E0EE0F59
:1069F000FF1FEB50F74FE080F180D7011296ED9129
:106A0000FC911397E4918E2F8023C1F1E1FF0AC01E
:106A10008CE0E7E7F7E0DE011D9601900D928A9584
:106A2000E1F706C0BE01635F7F4FC7010E94C43417
:106A3000A501BE01635F7F4F83E00E942116BE0166
:106A40006F5F7F4FC7010E947E329E01275E3F4FDE
:106A5000AE014F5F5F4FBA0183E00E944A07AE016B
:106A6000435F5F4FBE016F5F7F4F83E00E94191548
:106A7000882321F0F6011083C70106C01F5FB0CF45
:106A8000D6011C9380E090E06C960FB6F894DEBFC0
:106A90000FBECDBFDF91CF911F910F91FF90EF906F
:106AA000DF90CF90BF90AF900895DB018F939F93BD
:106AB0000E94D535BF91AF91A29F800D911DA39FDC
:106AC000900DB29F900D11240895991B79E004C098
:106AD000991F961708F0961B881F7A95C9F780951D
:106AE000089597FB072E16F4009407D077FD09D080
:106AF0000E94D03607FC05D03EF4909581959F4FBB
:106B00000895709561957F4F0895A1E21A2EAA1BF2
:106B1000BB1BFD010DC0AA1FBB1FEE1FFF1FA2174D
:106B2000B307E407F50720F0A21BB30BE40BF50B4A
:106B3000661F771F881F991F1A9469F760957095D3
:106B4000809590959B01AC01BD01CF010895052E64
:106B500097FB1EF400940E94BE3557FD07D00E949B
:106B6000853507FC03D04EF40C94BE355095409506
:106B7000309521953F4F4F4F5F4F089590958095E9
:106B8000709561957F4F8F4F9F4F0895A29FB001E1
:106B9000B39FC001A39F700D811D1124911DB29F51
:106BA000700D811D1124911D08950E94C635A59F69
:106BB000900DB49F900DA49F800D911D11240895F8
:106BC000689401C0E894F92FF12B12F00C9414365C
:106BD000A0E0B0E0EEEEF5E30C948636092E0594C5
:106BE00022F40E947036112392F4F0E80F26FFEF92
:106BF000E094F09400951095B094C094D094A19432
:106C0000BF0ACF0ADF0AEF0AFF0A0F0B1F0B0E9411
:106C10001F3607FC0E947036CDB7DEB7ECE00C944F
:106C2000A236689401C0E8948F929F92CF93DF932D
:106C30000E941F36DF91CF919F908F9008958824F6
:106C40009924F401E401B0E49F93AA279A158B04D8
:106C50009C04ED05FE05CF05D007A10798F4AD2FE4
:106C6000DC2FCF2FFE2FE92D982C892E982F872FE0
:106C7000762F652F542F432F322F2227B85031F70C
:106C8000BF9127C01B2EBF91BB27220F331F441F6C
:106C9000551F661F771F881F991F881C991CEE1FA0
:106CA000FF1FCC1FDD1FAA1FBB1F8A149B04EC050E
:106CB000FD05CE05DF05A007B10748F08A189B083F
:106CC000EC09FD09CE09DF09A00BB10B21601A9474
:106CD000E1F62EF49401AF01BE01CD01000C089540
:106CE000609570958095909530954095509521953B
:106CF0003F4F4F4F5F4F6F4F7F4F8F4F9F4F0895C5
:106D00002F923F924F925F926F927F928F929F92BB
:106D1000AF92BF92CF92DF92EF92FF920F931F93A9
:106D2000CF93DF93CDB7DEB7CA1BDB0B0FB6F8945A
:106D3000DEBF0FBECDBF09942A88398848885F849A
:106D40006E847D848C849B84AA84B984C884DF800B
:106D5000EE80FD800C811B81AA81B981CE0FD11DEF
:106D60000FB6F894DEBF0FBECDBFED0108950F93AF
:106D7000083090F0982F872F762F652F542F432FB0
:106D8000322F22270850F4CF220F331F441F551FE4
:106D9000661F771F881F991F0A95B2F70F910895F4
:106DA000AA1BBB1B51E107C0AA1FBB1FA617B70731
:106DB00010F0A61BB70B881F991F5A95A9F780954D
:0C6DC0009095BC01CD010895F894FFCF20
:106DCC000000E0FF000020000000C0FF0080400039
:0E6DDC000000FFFF00000100010B04001A0080
:00000001FF
